:0408000055EF35F08B
:08080800046ED8CF05F0E0CF2B
:1008100006F00001E9CF0CF0EACF07F0E1CF08F0D5
:10082000E2CF09F0D9CF0AF0DACF0BF0F3CF12F014
:10083000F4CF13F0FACF14F0F5CF15F0F6CF16F091
:10084000F7CF17F000C00EF001C00FF002C010F09B
:1008500003C011F0F2AA30EF04F0F2B496EF17F0F3
:100860000EC000F00FC001F010C002F011C003F084
:100870000CC0E9FF07C0EAFF078E08C0E1FF09C00E
:10088000E2FF0AC0D9FF0BC0DAFF12C0F3FF13C0AA
:10089000F4FF14C0FAFF15C0F5FF16C0F6FF17C02D
:1008A000F7FF045006C0E0FF05C0D8FF1000F76A4C
:1008B000BE0FF66E080EF7220900F5501200000177
:1008C00002030405060710111213141516171C1D38
:1008D0001E1F3E3F5E5F91929397E80FF66E080EE3
:1008E000F7220900F5501200F19D656B976BAB3A4A
:1008F00065FD0FF5F1DE0A8E4A785BBA214421448A
:1009000018130072FD87D9AC9B50997212E7AE6A3A
:1009100021EA29B2442D25C7B505B505E9140066BD
:10092000EF2B7163ADAB693FA9152725E3C41452C2
:100930002024ECDB703370332815000353EC34F8BB
:1009400041FF271DE3F2B5B6E687AC72C027B08839
:10095000E92FE92F9C1900F9C4CC37D936EBF5C93A
:100960005BDD386306F7E96F94DE60D7F993F9939E
:10097000151C0057455722F7C3220E25384D3C1F42
:100980009851CE72F1BC94CBBE85BE852E1D008FD2
:1009900008B6D1A229FF060E785EBFC870980189FB
:1009A0009F40E2568D218D21A91F006380F588E7C5
:1009B00050AD563B67908E9AF0E272AEB9CF211BD4
:1009C0003E473E47522100CFEB8FB5120267786A4F
:1009D000A5BF2993A84FD7C63ED2E835E9BFE9BFE6
:1009E0004A2600648E4D9039B7761BE339F1E20A4E
:1009F000E33FA5E8897A782EBA74BA74BA320075E2
:100A0000026A712CB9EFCF827F4397AD4F0992E113
:100A1000E2D353014CC44CC4213300F186B2525D81
:100A2000DAF6F66F12114D575FBC733BE735701065
:100A30009272927272330086CB43C993F71B94EA89
:100A4000D4D9229EB8E9DF0CCA721FA8A700A7005C
:100A5000DD7902AD13E4DB903631701420AC1DCA91
:100A6000715F64C9E7EC6E25AA2EAA2E5648057060
:100A7000518689D94A252BDB122518D93CD0FEF4A2
:100A8000C271DC2323872387CA5B058E526ED7424F
:100A9000BD3C86117012CBE242B42FFB1C04C8F897
:100AA0005D7F5D7FA36B055F834CB79EA5B491C549
:100AB000515B009789A72269654AFCCAD5F0D5F039
:100AC0006ACA05A83284EBD1E3C439E55C78211108
:100AD000CAFC9DC87C40B611CE4FCE4F7CF4056752
:100AE000AB8F89B37D4C2CB871CC16DB84EA560EE3
:100AF000398AF9941F8E1F8E28020627C22220945D
:100B000083DB225D8F2638CA30AB11028DD308B249
:100B1000C391C3919317067647529010F4678D1DC9
:100B20000D861214288D579C151C326B1F531F53B2
:100B30004ED907F73C5BBC2E2BE1EA614939B7D1AE
:100B4000689A6B54E15C27AFE267E267A3E007E3D2
:100B5000F1C7CB2B1EC8AD7D754A333570A7CACF00
:100B6000E451476C42124212CE5A08022BC305418F
:100B700037D09D95520F8CD0B79A677CFB094208FD
:100B80004A2F4A2FAD6408BEF68624B45DF4ACDD6E
:100B9000A164DCD298AD599154657313A4CCA4CC54
:100BA00007F708D489BD51BF79D10D7F0CB89833B0
:100BB000EDD4B0054136E69228E128E1A1510B1DA4
:100BC000C4F45C3E068B4E1F579C2E4BABCF58A9EE
:100BD0001DCA068217A017A0A2810B1A1E73EE3C35
:100BE000A42A00460803FC2DEAC441990539AF83C5
:100BF000B504B5041B880B788F21BB29A0B36526EB
:100C0000D1501FA443BFAF7D997B1B10F37BF37BB7
:100C100099B70B175B88739B1B884246C89584372E
:100C2000FBB4505CD2D8EC4B169C169C81020D791B
:100C3000CC8247B8C660295E372923DC76D4875436
:100C4000CD79E2DC272E272E07210D9791D99C190B
:100C50004F2B0D000C1342360A83A179DAEA788112
:100C6000850F850F0E3C0D91110F57004AAEB06AEB
:100C70003404BB32C36805045793B718D1FAD1FACC
:100C8000253C0DDF6C1EAA7A04B2EBB7DA514C2278
:100C90004BA6B23EA87FD0D8BEBBBEBB425D0D45C1
:100CA0005C9D105A41595DF447F5DE55A43065A8A6
:100CB0000FF0411824AD24AD65640D015546942F05
:100CC0002F21D508E7BD08864EA6F94CD2EEB549CE
:100CD0001221122156920D8FB564C1E4279BBA846C
:100CE000BBC5EC28CB0F07F2FD4DF6F5E503E50398
:100CF0008C970D561666FB810CC67DFC20A80A5108
:100D0000327D31C04323A7DD07560756C5970DB581
:100D1000DC17E63B8680B22F2817ECC3449B10C536
:100D20000F9F4D1CE026E02622CB0DAD2DA28F0F8C
:100D30006BEC5572BB1201230321BD33513EF143CD
:100D40006AE16AE1D90F0E925E457529EBB2A51BE7
:100D50005A9DF11DFF044C74A0F295AB4EEA4EEA89
:100D6000375C0E7372532C45837389D12602B69873
:100D7000158E0F278C5E2C2B3CA73CA7B9BB0E0110
:100D800055451F71BF7B28417F30D614C730E325FE
:100D900096AD84A7944F944F64D10E23937CA3F017
:100DA000E79D65A5612891A1C3EA5FA5B6D6E93C98
:100DB0002D752D7582090F576332A6DFC31D93B5BC
:100DC00088481FD8A9152FCA0B98F10615D015D041
:100DD0005C120F8C65CC5338E09001CB3AAB46B82F
:100DE0003ED650D24516B8687CE57CE5091B0FBAA3
:100DF000EF4E04966AE2BDBE4051A377E047305102
:100E000088C4C9F4B00AB00ABA2A0FAD83C164E835
:100E10008249D1A2ED6267B6AE2D8973BF6794296E
:100E2000388C388CF06B0F332378493A49F22B3CDD
:100E30003140208728B2F69685F12AB023642364D6
:100E400021DE0F5D36135A25661066722ADF891A75
:100E50001946C65B0A31BE7B09920992890710AF19
:100E6000E54AA8695CD17984D597EDA9F62ADFF91E
:100E70007B9C1FC8347D347D9D74118434E2D9ED90
:100E8000ADC8FD74462C16917CD1050FC8C6AFEDD8
:100E900031F731F7D3BA1162DA6D10F2808D9F7499
:100EA000CB3D80BB5A803DD9DFE0E21EEF43EF43EC
:100EB000F6CB119F0EC332F311A2BA09D74EF2D668
:100EC00038D148731C1C07CB98609860B1D511B11C
:100ED000FD9335EFF8018B58BB3BBCCC6B52E1194D
:100EE000087CF0EC2CDF2CDF74F111220365721406
:100EF000FAD416B5D2BDAD20DF1926F7D5FD69426B
:100F000099DC99DC251D1248162E72D02D91088F80
:100F100095B0E7448554A1164A44D29574027402F0
:100F20004E5712275B864AE3D2A97644AF553F3E1F
:100F30009480B4DBD9A373FE92A292A20963124CEF
:100F40005A6BD00409D550B5F47E24D1BE6E66A18B
:100F500083E0FDDC21612161EB6F122AEFA90F858F
:100F60007BF78B542703867C9D948398B24435CEBF
:100F7000914A914A5275127A2890787AD82B6EA0AD
:100F8000EA13AD716BD88C19481306DFD3ABD3AB22
:100F9000EC821299A6C6E39D4F78A944344DA5B3BF
:100FA0001CC533F1D5954C516F536F5364B7128400
:100FB00031633A66D0B501294F6695128D169BB6FE
:100FC000D6D256A3C33EC33E5AB912D883D5120215
:100FD000C43CAF0487C817AA7591DFAA012E0B6C19
:100FE00061D561D5ECC312BDEDEA5A41D580745D7F
:100FF000D7CABD792A7A42967F9EB5331583158369
:1010000076D312BF0AE454D0D798ABCBF78267DE11
:10101000DD49A1BCC4A7234CABCDABCDE1DA12783E
:101020001BEB9E19D49C851C1827318A29B52812E0
:10103000DEDDE66BFE90FE905FFD12C5C5FE54132B
:101040005AEC738EEA0CC42A2A3A800EB8680F89CB
:101050002BC62BC6597613433423CFB7C208CA1503
:101060008726D14340EA464481AD856A9DC59DC52A
:101070000F661425DC3ACA9533FC70F9C19A36DF45
:101080000271D99C821DAB927035703542AB155BF5
:10109000C49F6AD3D0A8876F9EBD0A7A5CC0EABF9E
:1010A000C01DB2CA118A118AF9E31573EA833B3C69
:1010B0008702B7182CBF3202BA884611C6593F8B37
:1010C000ED93ED93042716FEDBC2DB0E101208A190
:1010D0004B5DC46733795280FA408F97144F144F99
:1010E000822F1698E696DFC7FF1FE322339511AAD9
:1010F000374D06225CE43E3A944E944ED4F91140AA
:10110000D2D7C8BCDBC377CF1D5C8A556AF9DDFE38
:10111000399614ADEE1BEE1BC90113CE274BBF272A
:101120009527BAF73A6F132E3334898D48C3DD9B68
:10113000124F124F7CC00861BBC17D7EE98265A859
:10114000F6DE3978B95C0B0B586F201F754975496D
:1011500036CC06EF6AD962474D28D46E8E322DAE5A
:1011600095773328A1579E9867B467B493B707CA99
:10117000A3C9B6137F550C56D747156E93622FDC63
:10118000B85E13451A721A72D1F50DA01861C30129
:10119000E772464F1DF215526CC0A3231259D46D4D
:1011A000D301D3016EA005D86ED139A3E7FD1BEBA7
:1011B00040A0B5578EB347AC0A9F6FBAA0A8A0A8AD
:1011C00027990D502B7C4CD3F0EE1C7793FCB1B4D7
:1011D00090C47020779E3D323C6B3C6B079812891F
:1011E000D4E808923D97082D649FE9B9EFA4E45034
:1011F000BE76E192AD2BAD2B18580EFE2737F4F4D6
:10120000218660C91D4567BFBD21EA63B0721E56C5
:101210006C4B6C4B69BD11FB6B11835985911CF5AF
:10122000BE6406BADB400ACE1D4ED70CF141F14137
:10123000D1940F7B81CBBC63431AD82BA59140AED0
:10124000CFDDCA6A979489A8C030C0301AE7129AD5
:10125000FB136A6BF627FE8FFF03A416748275CF0B
:101260005D23052D03BC03BC53010E152123F74F4D
:101270005AF50FCDDB002FE1758BCE1C34A57E54C3
:1012800024792479FFA712B101BE1F64697A43D67D
:10129000BD620E5FC286F91B9A36CCA072BF72BFC8
:1012A000A4110D166A9993D3FFF3124B91B65F7D8B
:1012B000730CA2396592110E2B742B743429089C7F
:1012C00081F510ACCBB485138B2579A1AF096AFBEE
:1012D00004670D94E454E45406591056863BF3BA5F
:1012E0005D6EA6C3FF5104EE21F843B3775AE26E58
:1012F000EB1EEB1E0BE511FD019DCFF0D5FF5C5100
:10130000664F01FE7497291C5819C996F319F319F1
:10131000AA130D865377B9A930C5D0750761FC9F14
:101320007C7FA0A21F25B2F2BE67BE67015313E601
:10133000CFF2A83FBD056E5ADB42748B581D89AFB2
:10134000BE8431D59CB59CB5DE9412FA78A30EB656
:1013500042862D75D6EF2AC1EDF7EC718583271AE9
:101360001EBA1EBA378812183A999AD52BE5B78457
:10137000BC3DB6ED95459D17827AD33A7BDF7BDF86
:1013800037C713111ADA68F6F9E3F5A4B2427A8185
:101390008CD7A76D61F181BD5CB45CB4A31B0AA8B6
:1013A00030C7AE22B15AADAEBCE9DA7789202E0A39
:1013B000B67B096AF6D6F6D6B3030EBFA4CD2136A6
:1013C000812E0EF609BF61849D08D283E992BFDCAD
:1013D00093E393E35F600932DE50228720FB3501FF
:1013E000D117F53C515122D4E52B5CCF945794573B
:1013F0006F430D679BC5742C7193B31103C30DFD2F
:10140000CB1D8B2CF4C275D5A3D7A3D707370EFFFE
:10141000477F23D44E41C51475D14145960BF563E2
:10142000E52CCED4327D327D53D10E4B93085B81B7
:1014300018759802F18966C0F85B0923C70D032E61
:1014400068E768E731AE06F8DA9E82CC34423BB3F7
:10145000C6158321A326832EC98C03887C747C74D3
:10146000951C06B4FB8E2F11C892ABF1B488F365BE
:101470007CE09A0D75D9D1025F0D5F0DE0DC097F2C
:10148000F080FBE88CC44124B950FB1E1968E33995
:101490008218F2E7A4ABA4AB43C412942563315D78
:1014A0002050726F6772616D20426C61636B202007
:1014B0002020202020325D2050726F6772616D20E5
:1014C0004379616E202020202020202020335D20C1
:1014D00050726F6772616D204D6167656E74612037
:1014E00020202025630D0A002563345D2050726F93
:1014F0006772616D2059656C6C6F77202020202009
:1015000020355D2050726F6772616D204C2F4379DA
:10151000616E20202020202020365D2050726F67D1
:1015200072616D204C2F4D6167656E7461202025BE
:10153000630D0A0025632D2D2D2D2D2D2D2D2D2DE7
:101540002D2D2D2D2D2D2D2D2D2D2D2D2D2D2D2DCB
:101550002D2D2D2D2D2D2D2D2D2D2D2D2D2D2D2DBB
:101560002D2D2D2D2D2D2D2D2D2D2D2D2D2D2D2DAB
:101570002D2D2D2D2D2D2D2D2D2D2D25630D0A00DD
:101580002563415D20526561642055494420202037
:10159000202020202020202020425D2052656164F0
:1015A00020445332343331204D656D6F72792020E1
:1015B00020485D205265616420636F706965642016
:1015C0006461746120202025630D0A0025634E5D4F
:1015D00020436F707920612063686970202020208B
:1015E00020202020204F5D20506173746520746896
:1015F00065206368697020202020202020515D2014
:1016000050757263686173652043726564697473B1
:1016100020202025630D0A002563495D2053657451
:1016200020646576696365206461746520202020EC
:1016300020505D205365742050726F6772616D6D2C
:10164000696E67204D6F64652020202020202020B7
:101650002020202020202020202020202020202585
:10166000630D0A002563455D20526561642074683E
:1016700065205350202020202020202020465D205F
:1016800057726974652074686520535020202020AB
:101690002020202020475D20436F70792053502068
:1016A000746F204D656D6F7279202025630D0A00DF
:1016B00025634C5D2052657365742D41636B205426
:1016C000657374202020202020435D2053656172C3
:1016D00063682055494420202020202020202020FD
:1016E00020445D204D6174636820524F4D20546545
:1016F0007374202020202025630D0A002563595D86
:10170000204D656D6F72792064756D702852415758
:101710002920202020505D2056696577204372657E
:1017200064697473207374617475732020585D202C
:10173000446961676E6F73746963206D6F646520BF
:1017400020202025630D0A004675747572652054AB
:101750006563686E6F6C6F6769657300536F75744E
:10176000682041667269636100002B2B3237323189
:10177000203937362D35383131000D0A50726573F6
:101780007320616E79206B657920746F20636F6EB2
:1017900074696E75652E2E2E0000426C61636B209D
:1017A000202020202020202020004379616E20204E
:1017B000202020202020202020004D6167656E74AD
:1017C0006120202020202020200059656C6C6F773C
:1017D000202020202020202020004C6967687420D1
:1017E0004379616E2020202020004C6967687420B6
:1017F0004D6167656E74612020004D756C7469647D
:10180000726F70206D6F646520004E6F2063686991
:10181000702070726573656E7400556E64656669DC
:101820006E656420636F6C6F72002020202025633A
:101830000000202020202563204D61696E204D6529
:101840006E75202D20004D616E7566616374757232
:101850006520646174653A20000057617272656E9C
:1018600074656520656E64733A202020000025753C
:101870002F25752F254C753A202020205265706544
:10188000617420436F756E7465723A2D20254C7516
:101890000D0A000020202020204850383030302011
:1018A000496E6B204361727472696467652052658A
:1018B00073657474696E672F50726F6772616D6DB6
:1018C000696E6720446576696365205265762031CC
:1018D0002E31300D0A002020202020202020202022
:1018E0000000202D2054656C3A002E0D0A0A0000DD
:1018F0000D0A53656C656374206F7074696F6E3A7E
:101900002020000044657669636520536572696133
:101910006C204E756D6265723A256C75202D2052D3
:1019200065736574206C6F673A25750D0A0A0000AF
:1019300028506C65617365204E4F54453A20746899
:10194000652061626F766520696E666F726D617485
:10195000696F6E206D7573742062652071756F7488
:101960006564207768656E2070757263686173695D
:101970006E6720637265646974732E0D0A00546883
:10198000697320696E666F726D6174696F6E20692C
:1019900073207573656420746F2067656E6572616E
:1019A00074652061206B65792074686174207769A3
:1019B0006C6C2062652073656E74206261636B20BD
:1019C000746F20796F752E290D0A0A0043726564C1
:1019D0006974732072656D61696E696E673A20255E
:1019E0006C750D0A0A000D0A456E746572207468E4
:1019F00065206E756D626572206F66207265736515
:101A0000742063726564697473206265696E67200F
:101A10007075726368617365643A2D2020000D0A49
:101A2000456E746572207468652034302063686187
:101A3000726163746572206B6579636F646520738E
:101A40007570706C69656420627920003A2D200DF4
:101A50000A000D0A526573657420637265646974C7
:101A60007320616D6D656E64656420737563636575
:101A7000737366756C6C792066726F6D20256C755A
:101A800020746F20256C752E00000D0A496E76615A
:101A90006C696420636F64652E002A2A2A2A00007C
:101AA00052204520532045205400572052204920E1
:101AB00054204520202020502052204F20432045F4
:101AC0002053205300002020205320552043204342
:101AD0002045205320462055204C2A2A2A2A00003F
:101AE0000A0A0D524553455420636F756E74657232
:101AF0002069732061646A757374656420746F3A39
:101B000020256C750A0D00000D0A20284E6F2063F9
:101B10007265646974732072656D61696E696E6760
:101B20002E20507572636861736520637265646905
:101B300074732066726F6D2046542E290D0A0000C2
:101B400043415554494F4E2120596F75206F6E6C9B
:101B500079206861766520256C75206372656469FB
:101B600074002072656D61696E696E672E20507514
:101B7000726368617365206372656469747320665B
:101B8000726F6D200D0A0000206265666F7265201D
:101B9000796F7572206372656469747320636F7501
:101BA0006E7465722072656163686573207A657210
:101BB0006F2E00000D4552524F523A205468652056
:101BC000312D576972652062757320686173206ECC
:101BD0006F20766F6C7461676520737570706C79B7
:101BE00000000D4552524F523A205468652052452C
:101BF0005345542070756C7365206973206E6F7443
:101C0000206265696E672041434B6E6F776C656437
:101C1000676564000D5265747279696E672E2E20B7
:101C200020202020202020202020202020202020B4
:101C300020202020202020202020202020202020A4
:101C400020202020200046616D696C7920436F645C
:101C5000653A20253258202049443A20000020438C
:101C600052433A202532580D0A000D0A204E6F20AB
:101C700064657669636573206F6E207468652031D2
:101C80002D5769726520627573002532553A2D20F3
:101C900020002532553A2D2020000D0A4465766932
:101CA00063652F732070726573656E742C20627586
:101CB00074206E6F7420746865206D756C74692D66
:101CC00064726F70207661726965747900000D0A24
:101CD000456E74657220776869636820646576690B
:101CE00063652773206D656D6F7279206973207449
:101CF0006F20626520696E746572726F67617465CA
:101D0000642E20427920656E746572696E67206169
:101D1000206E756D626572206E6F74000D0A6C69BD
:101D2000737465642077696C6C2070726576656E7B
:101D300074206120737065636966696320646576E9
:101D4000696365206F6E20746865206D756C7469B9
:101D500064726F70206275732066726F6D206265A9
:101D6000696E67000D0A6163746976617465642E3B
:101D700020000D4552524F523A2054686520312DB3
:101D8000576972652062757320686173206E6F20D9
:101D9000766F6C7461676520737570706C79000084
:101DA0000D0A0A52657365743A25752041434B2725
:101DB000733A25750D0A00000D4552524F523A20D4
:101DC00054686520312D57697265206275732068EB
:101DD0006173206E6F20766F6C7461676520737518
:101DE00070706C7900000D0A0A52657365743A25AB
:101DF000752041434B27733A25750D0A00000D0AE3
:101E0000202020203030203031203032203033204C
:101E100030342030352030362030372030382030F4
:101E2000392030412030422030432030442030459A
:101E30002030460D0A000D0A2020202030302030AE
:101E400031203032203033203034203035203036CD
:101E500020303720303820303920304120304220A7
:101E600030432030442030452030460D0A000D0A12
:101E700020414820414C2045532020203030203044
:101E8000312030322030332030342030352030368D
:101E900020303720202020434820434C0D0A0000EA
:101EA0000D0A0A456E74657220746865207461724B
:101EB0006765742061646472657373206F66206D5A
:101EC000656D6F72792830783030207468727520B3
:101ED00030783846293A00000D0A456E7465722044
:101EE00038206279746573206F66206461746120A4
:101EF000746F20777269746528696E206865782927
:101F00003A000D0A535020646174612070726F674B
:101F100072616D6D65643A0D0A005363726174639A
:101F2000687061642070726F6772616D6D656420A6
:101F3000776974682074686520666F6C6C6F776968
:101F40006E6720646174610D0A0A000041482041F7
:101F50004C202020303020303120303220303320CF
:101F600030342030352030362030370D0A00203113
:101F7000366269742043524320646174613A0D0AE9
:101F80000000202046726F6D2063686970206465D0
:101F9000766963653A2D2020202025325825325855
:101FA0000D0A00002020436F6D7075746564206217
:101FB000792072657365747465723A2025325825EC
:101FC00032580D0A0A000D0A436F7079205363726C
:101FD0006174636870616420000053554343455346
:101FE0005346554C212100004641494C454421218E
:101FF00000000D0A496E707574206465766963652A
:10200000207965617228323030372074687275200B
:1020100032303137293A20000D0A496E707574202C
:10202000646576696365206D6F6E7468283120740D
:1020300068727520313229203A2000000D0A496E5D
:1020400070757420646576696365206461792831F0
:10205000207468727520333129203A2000000D0A5F
:1020600044617465206368616E676520737563639E
:1020700065737366756C6C2E0D0A000050726F6785
:1020800072616D6D65642063686970732077696C37
:102090006C206E6F7720636F6E7461696E20746858
:1020A000697320656E636F64656420646174652084
:1020B00076616C75652E202532582532580D0A0040
:1020C0000D0A436F7079696E672074686520696DC9
:1020D0006167652066726F6D20746865206368694A
:1020E00070200D0A0A000D0A4E6F7720636F707919
:1020F000696E6720616464726573733A2D20000015
:102100000D0A0A436F707920636F6D706C6574659A
:10211000642E2E2E2E0D0A000D0A41646472657322
:10212000732070726F6772616D6D65643A20000094
:102130002532583A25325820253258202A2A2000A4
:102140000D0A4E6F20637265646974732072656D49
:1021500061696E696E672E2E2E000D0A41646472ED
:102160006573732070726F6772616D6D65643A207C
:102170000000030E0101F75F0BE3010EEA6EF70E9C
:10218000E96EEF5005E002D000000400EF2EFCD70E
:102190000001000C93908A900400030E0101F06F7F
:1021A000F20EF76F0001E5DF0101F02FF9D7938000
:1021B0000400070E006E002EFED700D0938081B081
:1021C00003D0000E016E19D004006B0E006E002EBD
:1021D000FED700D09380EF9181A0EF810400EF0E35
:1021E000F76F0001C6DF0101EFA104D0010E016EFF
:1021F00004D003D0000E016E00D0000199EF17F05B
:102200001B0E04009EA8FDD7AD6E5B0E04009EA8B9
:10221000FDD7AD6E320E04009EA8FDD7AD6E4A0EFE
:1022200004009EA8FDD7AD6E000C0900F5520EE02B
:10223000F6CF00F2F7CF01F2F55004009EA8FDD7CB
:10224000AD6E00C2F6FF01C2F7FFEFD7000C02012E
:102250000351016A025D03E202C200F00CD0006A81
:10226000080E046F023700360351005CD8B0006ED0
:102270000136042FF7D70001000C015000C202F212
:10228000640E0201036F0001E2DF00C000F20150A2
:10229000300E08E1020101A30FD001B70DD001B942
:1022A000200E04D0020101970199018101260150FD
:1022B00004009EA8FDD7AD6E00C202F20A0E036FA5
:1022C0000001C5DF00C000F20150300E08E102013C
:1022D00001B70CD001A10AD001B9200E00010126DE
:1022E000015004009EA8FDD7AD6E0201300E0027FC
:1022F000005104009EA8FDD7AD6E0001000CEACF8E
:1023000006F2E9CF05F20101FE39F0090201016F81
:102310000127E20F026F320F046F0101FE510F0B14
:102320000201022702270427E90F036F032703276F
:102330000101FD390F0B020103270427033704377E
:10234000041F04370101FD510F0B0201042701375F
:10235000070E006F0A0E03070427FDE30207032799
:10236000FDE301070227FDE300070127FDE3020E5D
:10237000EA6EE96A070E0515059DE926040EE95C7B
:10238000D8B4058DEF50006E08E105BD06D005B943
:102390000DD005B702D0200E03D005870599300E69
:1023A0000026005004009EA8FDD7AD6EEE5005AD8E
:1023B000E5D70001000C0900F6CF01F2F7CF02F2D9
:1023C000F55004009EA8FDD7AD6E01C2F6FF02C213
:1023D000F7FF0201002F01D002D00001ECD700016D
:1023E000000C0101F5511F0BF96FF631FE6FF5314D
:1023F000FD6FFE33FD33FE33FD33FE33FD33FE331D
:10240000FD33070EFE17FD510F0BFA6FD890FE6BD0
:10241000F631FD6FD00EFD25FB6F070EFE21FC6F20
:10242000F85308E1460EF66E180EF76E0001FDDE59
:102430000AD001015A0EF66E180EF76E0001F5DE95
:10244000010E0101F95F0101F7533AE0F9C100F211
:102450001B0E0201016F000110DF2F0E04009EA869
:10246000FDD7AD6EFAC100F21B0E0201016F000133
:1024700004DF2F0E04009EA8FDD7AD6E100EE96E8E
:10248000FCC1FEF1FBC1FDF13ADF770EF66E180ECE
:10249000F76E160E0201006F00018DDF100EE96E5F
:1024A000D8C0FEF1D7C0FDF12ADF0D0E04009EA8B2
:1024B000FDD7AD6E0A0E04009EA8FDD7AD6E29D0E3
:1024C000F9C100F21B0E0201016F0001D6DE2F0ED2
:1024D00004009EA8FDD7AD6EFAC100F21B0E0201EA
:1024E000016F0001CADE2F0E04009EA8FDD7AD6E5D
:1024F000100EE96EFCC1FEF1FBC1FDF100DF0D0E17
:1025000004009EA8FDD7AD6E0A0E04009EA8FDD75C
:10251000AD6E000C0101F451000A00010FE0010A48
:1025200013E0030A17E0010A1BE0070A1FE0010A93
:1025300023E0FB0A27E0010A2BE030D09A0EF66E6A
:10254000170EF76E72DE30D0AA0EF66E170EF76E0B
:102550006CDE2AD0BA0EF66E170EF76E66DE24D049
:10256000CA0EF66E170EF76E60DE1ED0DA0EF66E2D
:10257000170EF76E5ADE18D0EA0EF66E170EF76ECB
:1025800054DE12D0FA0EF66E170EF76E4EDE0CD039
:102590000A0EF66E180EF76E48DE06D01A0EF66EAC
:1025A000180EF76E42DE00D0000C2A0EF66E180EE2
:1025B000F76E040E0201006F0001FDDEC90E04007B
:1025C0009EA8FDD7AD6E0101EF6BEF513B0807E30D
:1025D000CD0E04009EA8FDD7AD6EEF2BF6D7BB0E37
:1025E00004009EA8FDD7AD6E0D0E04009EA8FDD779
:1025F000AD6E0A0E04009EA8FDD7AD6E320EF66ECB
:10260000180EF76E040E0201006F0001D4DEBA0E40
:1026100004009EA8FDD7AD6E380EF66E180EF76E4C
:102620000D0E0201006F0001C6DEBCC0F4F172DFC6
:102630000101EF6BEF511F0807E3200E04009EA875
:10264000FDD7AD6EEF2BF6D7BA0E04009EA8FDD7CE
:10265000AD6E0D0E04009EA8FDD7AD6E0A0E0400EF
:102660009EA8FDD7AD6EDA0E04009EA8FDD7AD6E14
:10267000C40E04009EA8FDD7AD6EC40E04009EA833
:10268000FDD7AD6EC40E04009EA8FDD7AD6ED00E72
:1026900004009EA8FDD7AD6EEF6BEF513B0807E33A
:1026A000C40E04009EA8FDD7AD6EEF2BF6D7D00E5A
:1026B00004009EA8FDD7AD6EEF6BEF51030807E352
:1026C000C40E04009EA8FDD7AD6EEF2BF6D7BF0E4B
:1026D00004009EA8FDD7AD6E0D0E04009EA8FDD788
:1026E000AD6E0A0E04009EA8FDD7AD6EB30E0400B9
:1026F0009EA8FDD7AD6E9E0EF66E140EF76E450EBB
:102700000201006F000157DEB30E04009EA8FDD742
:10271000AD6E0D0E04009EA8FDD7AD6E0A0E04002E
:102720009EA8FDD7AD6EB30E04009EA8FDD7AD6E7A
:10273000EA0EF66E140EF76E450E0201006F0001F0
:102740003ADEB30E04009EA8FDD7AD6E0D0E040058
:102750009EA8FDD7AD6E0A0E04009EA8FDD7AD6EF3
:10276000B30E04009EA8FDD7AD6E360EF66E150EA4
:10277000F76E450E0201006F00011DDEB30E04006E
:102780009EA8FDD7AD6E0D0E04009EA8FDD7AD6EC0
:102790000A0E04009EA8FDD7AD6EB30E04009EA8DD
:1027A000FDD7AD6E820EF66E150EF76E450E020168
:1027B000006F000100DEB30E04009EA8FDD7AD6ED1
:1027C0000D0E04009EA8FDD7AD6E0A0E04009EA853
:1027D000FDD7AD6EB30E04009EA8FDD7AD6ECE0E34
:1027E000F66E150EF76E450E0201006F0001E3DD77
:1027F000B30E04009EA8FDD7AD6E0D0E04009EA87A
:10280000FDD7AD6E0A0E04009EA8FDD7AD6EB30EC7
:1028100004009EA8FDD7AD6E1A0EF66E160EF76E6A
:10282000450E0201006F0001C6DDB30E04009EA834
:10283000FDD7AD6E0D0E04009EA8FDD7AD6E0A0E3D
:1028400004009EA8FDD7AD6EBBA13AD0B30E040024
:102850009EA8FDD7AD6E660EF66E160EF76E450E8F
:102860000201006F0001A7DDB30E04009EA8FDD792
:10287000AD6E0D0E04009EA8FDD7AD6E0A0E0400CD
:102880009EA8FDD7AD6EB30E04009EA8FDD7AD6E19
:10289000B20EF66E160EF76E450E0201006F0001C5
:1028A0008ADDB30E04009EA8FDD7AD6E0D0E0400A8
:1028B0009EA8FDD7AD6E0A0E04009EA8FDD7AD6E92
:1028C000B30E04009EA8FDD7AD6EFE0EF66E160E7A
:1028D000F76E450E0201006F00016DDDB30E0400BE
:1028E0009EA8FDD7AD6E0D0E04009EA8FDD7AD6E5F
:1028F0000A0E04009EA8FDD7AD6EC00E04009EA86F
:10290000FDD7AD6E0101EF6BEF51440807E3C40E34
:1029100004009EA8FDD7AD6EEF2BF6D7D90E0400AC
:102920009EA8FDD7AD6E0001000C6ADC940EF66E19
:10293000180EF76E7ADCD60EF66E180EF76E75DC92
:10294000480EF66E170EF76E70DC2E0E04009EA871
:10295000FDD7AD6E200E04009EA8FDD7AD6E5C0EB7
:10296000F66E170EF76E61DCE20EF66E180EF76E5D
:102970005CDC6A0EF66E170EF76E57DCEA0EF66E2A
:10298000180EF76E52DC200E04009EA8FDD7AD6E27
:10299000200E04009EA8FDD7AD6EF2CFEFF1F29E9F
:1029A000AA6A130EA96EA69CA69EA680A850010135
:1029B000EFBFF28EF06FF2CFF1F1F29EAA6A140E21
:1029C000A96EA69CA69EA680A850F1BFF28EF26FBB
:1029D000F0C1F4F1F2C1F3F1F4C1F6F1F3C1F5F194
:1029E000010EF76FF86B0001FCDC0A0E04009EA8D4
:1029F000FDD7AD6EDADDF00EF66E180EF76E15DC53
:102A0000000C010EEA6EF80EE96EEF5011E0060EB2
:102A1000016EBF0E006E0400002EFDD7012EF9D707
:102A20007A0E006E002EFED700D00400EF2EEFD7F6
:102A3000000C93908A900400030E0101F66FF20ED1
:102A4000F76F0001B9EC10F00101F62FF8D7938071
:102A50000400070E006E002EFED700D0938081B0D8
:102A600014D0B40EF66E1B0EF76E000115EC11F0CB
:102A7000020E0101F66FFA0EF86F0001C2DF0101CC
:102A8000F62FF9D7000E016E3CD004006B0E006EDD
:102A9000002EFED700D09380F59181A0F58104002F
:102AA000EF0EF76F0001B9EC10F00101F5A104D0B1
:102AB000010E016E26D025D0E20EF66E1B0EF76ECB
:102AC000000115EC11F0020E0101F66FFA0EF86F1D
:102AD000000197DF0101F62FF9D7140EF66E1C0ED8
:102AE000F76E000115EC11F0020E0101F66FFA0EFF
:102AF000F86F000186DF0101F62FF9D7000E016E95
:102B000000D00001000C010E0101F76FF751080819
:102B10002FE393908A90D890F6330EE393908A80B7
:102B20000400200E006E002EFED700D081B003D02E
:102B3000000E016E1FD00DD093908A900400200EDD
:102B4000006E002EFED700D081A003D0000E016ED3
:102B500011D00400330E006E002EFED793908A80B1
:102B60000400070E006E002EFED700D0F72BCED744
:102B7000010E016E0001000C5CDF0152FDE004005B
:102B8000020E0101F56FD10EF76F0001B9EC10F0E4
:102B90000101F52FF8D7550EF66F0001B4DF0400E0
:102BA000060E006E002EFED70101F46BF4510708EB
:102BB0001FE30400060E006E002EFED73D51080DE7
:102BC000F350F66BF56F036AF451F525016EF6517B
:102BD00003220150ED0FE96E000E0320EA6EEFCFE5
:102BE000F5F1F5C1F6F100018EDF0101F42BDED71E
:102BF0000001000C010E0101F66FF651080820E3F8
:102C000093908A9093800400200E006E002EFED7D1
:102C100000D0938081B002D0D89001D0D880F73313
:102C200004003B0E006E002EFED70000F651030894
:102C300005E1C80EF86F0001E4DE0101F62BDDD7D7
:102C4000F7C101F00001000C010E0101F66FF65111
:102C5000080818E393908A9093800400200E006E79
:102C6000002EFED700D0938081B002D0D89001D042
:102C7000D880F73304003B0E006E002EFED7000014
:102C8000F62BE5D7F7C101F00001000C0101F6BFFA
:102C900011D00F0E006EF53900160A0E005C03E22B
:102CA000300E002602D0F6510026005004009EA8E7
:102CB000FDD7AD6E0F0EF5170A0EF55D02E2300E70
:102CC00002D0F69FF651F527F55104009EA8FDD7D6
:102CD000AD6E0001000C0101F053D8A46FD03D3D52
:102CE00001D004D0000148DF15D001010001A1DEB0
:102CF0000152FDE00400020E0101F46FD10EF76FE6
:102D00000001B9EC10F00101F42FF8D7CC0EF66FEA
:102D10000001F9DE0400060E006E002EFED7F00E54
:102D20000101F66F0001EFDE0400060E006E002EBA
:102D3000FED70101F66B0001E6DE0400060E006E10
:102D4000002EFED70101F66B0001DDDE0101F16B03
:102D5000F1518F0832E30400040E006E002EFED7FE
:102D60000000F151050814E1036AF1511E0F016ED4
:102D7000000E032201C0F4F103C0F5F100013ADFB7
:102D8000F5C1EAFFF4C1E9FF01C0EFFF13D0010173
:102D9000036AF1511E0F016E000E032201C0F4F10F
:102DA00003C0F5F1000150DFF5C1EAFFF4C1E9FF0E
:102DB00001C0EFFF0101F12BCBD71FD0F16BF15117
:102DC0008F081BE3036AF1511E0FE96E000E03200A
:102DD000EA6EF151F66F010EF76FF2CFF8F1F29E45
:102DE000F7C1AAFFF6C1A9FFA69CA69EA680A8507F
:102DF000F8BFF28EEF6EF12BE2D7EF53D8B479D053
:102E0000FE0EF66E1D0EF76E000115EC11F00101BD
:102E1000F16BF1518F0858E3F1510F0B3EE1F15185
:102E200080080AE10D0E04009EA8FDD7AD6E0A0EC3
:102E300004009EA8FDD7AD6E036AF1511E0FE96E26
:102E4000000E0320EA6EEFCFF4F10D0E04009EA8F1
:102E5000FDD7AD6E0A0E04009EA8FDD7AD6EF1C180
:102E6000F5F1370EF66F000111DF200E04009EA869
:102E7000FDD7AD6E200E04009EA8FDD7AD6EF4C147
:102E8000F5F1370E0101F66F000100DF200E04009E
:102E90009EA8FDD7AD6E15D00101036AF1511E0F3A
:102EA000E96E000E0320EA6EEFCFF4F1F4C1F5F104
:102EB000370EF66F0001EADE200E04009EA8FDD753
:102EC000AD6E0101F12BA5D726C0F4F100018AEC0B
:102ED00012F00D0E04009EA8FDD7AD6E0A0E040080
:102EE0009EA8FDD7AD6E0A0E04009EA8FDD7AD6E5C
:102EF00001012CC0F3F12DC0F2F1F3C1F6F1F2C1E2
:102F0000F5F1F76BF86B0001F1EC11F086C0F3F10D
:102F100087C0F2F1F3C1F6F1F2C1F5F10101F76BEF
:102F2000010EF86F0001F1EC11F0000C0400CAEF83
:102F300010F001520CE10400FF0EBC6FBB93BD51B9
:102F4000BC5D03E0F2DCBCC0BDF011D010D0BBB35F
:102F500005D00101EF6BF06B0001BDDEBB8326C025
:102F6000BCF0BD51BC5D03E0BCC0BDF0DEDCF29442
:102F700030EF04F092908990000C9280000C9382C4
:102F800093968A96938493988A98939A8A9AC5EF8F
:102F900035F00101E351E503F3CF01F0F4CF00F088
:102FA000E603F3500026E451E503F3500020026EDF
:102FB0000001000C1B0E04009EA8FDD7AD6E5B0E39
:102FC00004009EA8FDD7AD6E730E04009EA8FDD729
:102FD000AD6E000C1B0E04009EA8FDD7AD6E5B0EFF
:102FE00004009EA8FDD7AD6E750E04009EA8FDD707
:102FF000AD6E000C0101E56BE46BE35304E00001EE
:1030000000EC11F00101F2CFE6F1F29EAA6A100E77
:10301000A96EA69CA69EA680A850E6BFF28EE76F7A
:10302000F2CFE8F1F29EAA6A110EA96EA69CA69EA6
:10303000A680A850E8BFF28EE96FE7C1E5F1E9C1CB
:10304000E4F1E551260837E2FF0A03E1E4511008F4
:1030500032E2E56B320EE46FE5C1E6F1E76BAA6A96
:10306000100EA96EE6C1A8FFA69CA69EA684F250EB
:10307000006EF29E0F01550EA76EAA0EA76EA682D5
:10308000A6B2FED7A6940050F212AA6A110EA96E3B
:10309000E4C1A8FFA69CA69EA684F2CF00F0F29EF3
:1030A000550EA76EAA0EA76EA682A6B2FED7A6944C
:1030B0000050F2120101E151E45F000EE55BE5C151
:1030C000E6F1E76BAA6A100EA96EE6C1A8FFA69CFE
:1030D000A69EA684F250006EF29E0F01550EA76EBA
:1030E000AA0EA76EA682A6B2FED7A6940050F21230
:1030F000AA6A110EA96EE4C1A8FFA69CA69EA6848A
:10310000F2CF00F0F29E550EA76EAA0EA76EA68211
:10311000A6B2FED7A6940050F2129A0EF66E1A0EC0
:10312000F76E196AF2BE198EF29E000115EC11F0CD
:1031300019BEF28E0101E2530FE1A00EF66E1A0ED7
:10314000F76E196AF2BE198EF29E000115EC11F0AD
:1031500019BEF28E0ED00101AA0EF66E1A0EF76E8F
:10316000196AF2BE198EF29E000115EC11F019BE1B
:10317000F28EC60EF66E1A0EF76E196AF2BE198E30
:10318000F29E15EC11F019BEF28EE00EF66E1A0EDC
:10319000F76E196AF2BE198EF29E210E0201006FBF
:1031A0000001DBEC11F019BEF28E100EE96E196A07
:1031B000F2BE198EF29EE5C1FEF1E4C1FDF17FEC95
:1031C00011F019BEF28E0A0E04009EA8FDD7AD6E56
:1031D0000D0E04009EA8FDD7AD6E080E0101E66F2E
:1031E000196AF2BE198EF29EFA0EF86F000109DC20
:1031F00019BEF28E0101E62FF3D70001000C010188
:10320000426B436B446B456B466B476B486B496B3A
:103210004A6B0B0E4B6FFF0E4C6F4D6B110E4E6FCA
:10322000020E4F6F120E506FCB0E516F526B536BDD
:10323000546B556B566B576B586B596B5A6B070E2B
:103240005B6FA10E5C6F200E5D6FC00E5E6F270E70
:103250005F6FB00E606F880E616F626B636BFF0E05
:10326000646F656B666B676B686B696B6A6B6B6BC6
:103270006C6B6D6B6E6F6F6F706F716F726F736F62
:10328000746F756F766F776F786F796F7A6F7B6F0A
:103290007C6F7D6F7E6F7F6FE90E806F2F0E816F69
:1032A000826B836BFF0E846F856B866B876B886B7D
:1032B000896B8A6B8B6B8C6B8D6B8E6F8F6F906F46
:1032C000916F926F936F946F956F966F976F986FE2
:1032D000996F9A6F9B6F9C6F9D6F9E6F9F6FE90EAA
:1032E000A06F2F0EA16FA26BA36B220EA46FC40E52
:1032F000A56F120EA66FCB0EA76F120EA86FCB0E86
:10330000A96F140EAA6FEB0EAB6FFF0EAC6FAD6F13
:10331000AE6FAF6FB06FB16FB26FB36FB46FB56FA9
:10332000B66FB76FB86FB96FBA6FBB6FBC6FBD6F59
:10333000BE6FBF6FC06FC16FC26BC36BC46BAA0E91
:10334000C56FC66B550EC76FC86B0A0EC96FCA6BC7
:10335000CB6BCC6BCD6BCE6BCF6B010ED06F0A0EEF
:10336000D16FAD0ED26FD36BD46BD56B100ED66F01
:10337000300ED76F100ED86FD96BDC6BE06BDF6B44
:10338000F2CFE1F1F29EAA6A100EA96EA69CA69E4B
:10339000A680A850E1BFF28EE26FF2CFE3F1F29E79
:1033A000AA6A110EA96EA69CA69EA680A850E3BF8D
:1033B000F28EE46FE2C1E0F1E4C1DFF1DF5321E11D
:1033C000E0531FE1400EF66E210EF76E196AF2BE51
:1033D000198EF29E000115EC11F019BEF28E080E46
:1033E0000101E16F196AF2BE198EF29EFA0EF86FB2
:1033F000000101EC15F019BEF28E0101E12FF2D7A8
:103400009DD34151FA0FD8B027D2060F0001A0EF8B
:103410001DF001014A6BF2CFE1F1F29EAA6A400E63
:10342000A96EA69CA69EA680A850E1BFF28EDB6F77
:10343000DB516A0802E2DB6B01D0DB2BAA6A400E8B
:10344000A96EDBC1A8FFA69CA69EA684F250006EC2
:10345000F29E0F01550EA76EAA0EA76EA682A6B207
:10346000FED7A6940050F2120101DA6BDA511B0864
:1034700029E3036ADA51000157EC04F0036A420FB2
:10348000E96E010E0320EA6E0101E46BDBC1E3F19A
:10349000E66B1C0EE56F00017CDD02C0E4F101C0AB
:1034A000E3F10101DA510124016E000E0220036EE6
:1034B000015003C0F7FF00016DEC04F0EF6E010155
:1034C000DA2BD4D7C9D1010E01014A6FF2CFE1F155
:1034D000F29EAA6A400EA96EA69CA69EA680A8503F
:1034E000E1BFF28EDB6FDB516A0802E2DB6B01D0D9
:1034F000DB2BAA6A400EA96EDBC1A8FFA69CA69E84
:10350000A684F250006EF29E0F01550EA76EAA0E11
:10351000A76EA682A6B2FED7A6940050F2120101B1
:10352000DA6BDA511B0829E3036ADA51000157EC20
:1035300004F0036A420FE96E010E0320EA6E0101F6
:10354000E46BDBC1E3F1E66B1C0EE56F000121DDEE
:1035500002C0E4F101C0E3F10101DA510124016E7E
:10356000000E0220036E015003C0F7FF00016DEC56
:1035700004F0EF6E0101DA2BD4D76ED1020E0101F7
:103580004A6FF2CFE1F1F29EAA6A400EA96EA69CA4
:10359000A69EA680A850E1BFF28EDB6FDB516A08C1
:1035A00002E2DB6B01D0DB2BAA6A400EA96EDBC105
:1035B000A8FFA69CA69EA684F250006EF29E0F0164
:1035C000550EA76EAA0EA76EA682A6B2FED7A69427
:1035D0000050F2120101DA6BDA511B0829E3036A89
:1035E000DA51000157EC04F0036A420FE96E010E54
:1035F0000320EA6E0101E46BDBC1E3F1E66B1C0E14
:10360000E56F0001C6DC02C0E4F101C0E3F1010195
:10361000DA510124016E000E0220036E015003C036
:10362000F7FF00016DEC04F0EF6E0101DA2BD4D747
:1036300013D1030E01014A6FF2CFE1F1F29EAA6AA3
:10364000400EA96EA69CA69EA680A850E1BFF28E51
:10365000DB6FDB516A0802E2DB6B01D0DB2BAA6A6D
:10366000400EA96EDBC1A8FFA69CA69EA684F250C0
:10367000006EF29E0F01550EA76EAA0EA76EA682CF
:10368000A6B2FED7A6940050F2120101DA6BDA510D
:103690001B0829E3036ADA51000157EC04F0036ABE
:1036A000420FE96E010E0320EA6E0101E46BDBC1FB
:1036B000E3F1E66B1C0EE56F00016BDC02C0E4F188
:1036C00001C0E3F10101DA510124016E000E022074
:1036D000036E015003C0F7FF00016DEC04F0EF6EC4
:1036E0000101DA2BD4D7B8D0040E01014A6FF2CF12
:1036F000E1F1F29EAA6A400EA96EA69CA69EA68043
:10370000A850E1BFF28EDB6FDB516A0802E2DB6B8F
:1037100001D0DB2BAA6A400EA96EDBC1A8FFA69CD4
:10372000A69EA684F250006EF29E0F01550EA76E63
:10373000AA0EA76EA682A6B2FED7A6940050F212D9
:103740000101DA6BDA511B0829E3036ADA5100013F
:1037500057EC04F0036A420FE96E010E0320EA6E93
:103760000101E46BDBC1E3F1E66B1C0EE56F0001C8
:1037700010DC02C0E4F101C0E3F10101DA510124DF
:10378000016E000E0220036E015003C0F7FF00011E
:103790006DEC04F0EF6E0101DA2BD4D75DD0050E8D
:1037A00001014A6FF2CFE1F1F29EAA6A400EA96EC2
:1037B000A69CA69EA680A850E1BFF28EDB6FDB51CF
:1037C0006A0802E2DB6B01D0DB2BAA6A400EA96E0D
:1037D000DBC1A8FFA69CA69EA684F250006EF29EB6
:1037E0000F01550EA76EAA0EA76EA682A6B2FED72F
:1037F000A6940050F2120101DA6BDA511B082AE399
:10380000036ADA51000157EC04F0036A420FE96ED3
:10381000010E0320EA6E0101E46BDBC1E3F1E66B0C
:103820001C0EE56F0001C9EC17F002C0E4F101C005
:10383000E3F10101DA510124016E000E0220036E52
:10384000015003C0F7FF00016DEC04F0EF6E0101C1
:10385000DA2BD3D701D00101900EDD6FDD51960830
:103860002AE3DA6BDA51070824E3036ADD51420FD9
:10387000E96E010E0320EA6EEFCFE1F1E1C100F045
:10388000DA51016E04E0D8900032012EFCD7000E10
:1038900000B0010EE16F000EDCB1010EE11905E090
:1038A000D890DC338C0EDC1B02D0D890DC33DA2BC2
:1038B000D9D7DD2BD3D7DCC1D9F1F2CFE1F1F29E1C
:1038C000AA6A130EA96EA69CA69EA680A850E1BF68
:1038D000F28E506FF2CFE1F1F29EAA6A140EA96E39
:1038E000A69CA69EA680A850E1BFF28E516FF2CF93
:1038F000E1F1F29EAA6A130EA96EA69CA69EA6806E
:10390000A850E1BFF28EA66FF2CFE1F1F29EAA6A53
:10391000140EA96EA69CA69EA680A850E1BFF28EAA
:10392000A76FF2CFE1F1F29EAA6A130EA96EA69CD0
:10393000A69EA680A850E1BFF28EA86FF2CFE1F15B
:10394000F29EAA6A140EA96EA69CA69EA680A850F6
:10395000E1BFF28EA96F020EA825AA6F010EA9255C
:10396000AB6F5A0EF66E210EF76E196AF2BE198E03
:10397000F29E000115EC11F019BEF28EDAEC17F090
:10398000196AF2BE198EF29E19EC15F019BEF28E6C
:103990000152F6E0196AF2BE198EF29E990E0101EB
:1039A000F66F000183EC15F019BEF28E0400200EB4
:1039B000006E002EFED700D00101DA6BDA519708B5
:1039C000D8A0A3D0036ADA51420FE96E010E03209A
:1039D000EA6EEFCFE1F1196AF2BE198EF29EDAC1FA
:1039E000F5F1370EF66F000146EC16F019BEF28EB7
:1039F0003A0E04009EA8FDD7AD6E196AF2BE198E6C
:103A0000F29EE1C1F5F1370E0101F66F000146ECBF
:103A100016F019BEF28E200E04009EA8FDD7AD6EE2
:103A20002D0E04009EA8FDD7AD6E036A0101DA5188
:103A3000420FE96E010E0320EA6EEFCFE1F1196A41
:103A4000F2BE198EF29EE1C1F6F1000183EC15F091
:103A500019BEF28E0400100E006E002EFED7196AF9
:103A6000F2BE198EF29E24EC16F019BEF28E01C041
:103A7000DEF10400100E006E002EFED7036A010175
:103A8000DA51420FE96E010E0320EA6EEF50DE5D5F
:103A900031E1196AF2BE198EF29E770EF66F0001BF
:103AA00083EC15F019BEF28EEAEC17F0196AF2BE3B
:103AB000198EF29EDAC1F5F1370E0101F66F0001A1
:103AC00046EC16F019BEF28E196AF2BE198EF29EFD
:103AD000040E0101F86F000101EC15F019BEF28E21
:103AE000196AF2BE198EF29E24EC16F019BEF28EFF
:103AF00009D001010400200E006E002EFED700D078
:103B000061D700010101DA2B59D7010EE16FE26B99
:103B1000E36F0001FAEC17F0BB93080E0101E16FAF
:103B2000196AF2BE198EF29EFA0EF86F000101ECCE
:103B300015F019BEF28E0101E12FF2D70001000C41
:103B4000E824F76AF7365B0FF66E3B0EF7220A00A1
:103B5000F550FA6E0800F550F96E1234C6347C3513
:103B60003236E8369E37010145530AE00D0E040057
:103B70009EA8FDD7AD6E0A0E04009EA8FDD7AD6EBF
:103B8000460EF66E1C0EF76E196AF2BE198EF29E84
:103B90000D0E0201006F0001DBEC11F019BEF28E78
:103BA000196AF2BE198EF29ECFC0F5F1370E0101EF
:103BB000F66F000146EC16F019BEF28E560EF66E48
:103BC0001C0EF76E196AF2BE198EF29E060E0201E5
:103BD000006F0001DBEC11F019BEF28E010E010145
:103BE000466F465106081EE3036A4651CF0FE96E41
:103BF000000E0320EA6EEFCF47F1196AF2BE198E6C
:103C0000F29E47C1F5F1370EF66F000146EC16F053
:103C100019BEF28E200E04009EA8FDD7AD6E0101E4
:103C2000462BDFD75E0EF66E1C0EF76E196AF2BEDB
:103C3000198EF29E060E0201006F0001DBEC11F0FE
:103C400019BEF28E196AF2BE198EF29ED6C0F5F137
:103C5000370E0101F66F000146EC16F019BEF28E28
:103C60000D0E04009EA8FDD7AD6E0A0E04009EA89E
:103C7000FDD7AD6E000C196AF2BE198EF29E19ECDA
:103C800015F019BEF28E0152F6E00400020E010199
:103C9000436F196AF2BE198EF29ED10EF76F0001C2
:103CA000B9EC10F019BEF28E0101432FF2D7196A58
:103CB000F2BE198EF29E330EF66F000183EC15F002
:103CC00019BEF28E0101426B4251070821E3040044
:103CD000060E006E002EFED7036A4251CF0F016E12
:103CE000000E032201C043F103C044F1196AF2BE81
:103CF000198EF29E000124EC16F019BEF28E44C11A
:103D0000EAFF43C1E9FF01C0EFFF0101422BDCD70D
:103D1000415305E041C145F1000125DF01010001EA
:103D20001AEF37F07A0EF66E170EF76E196AF2BEBA
:103D3000198EF29E15EC11F019BEF28E04009EAAA7
:103D4000FDD7AE50000C04009EA8FDD7AD6E000C50
:103D500001016407656B04009EAAFDD7AECF66F132
:103D6000665108080EE165530BE0650766510001D6
:103D7000EADF200EE8DF010166510001E4DF010106
:103D800017D066511F0814E266517E0811E3655191
:103D9000645D0EE36551652B036A6225E96E63512C
:103DA0000320EA6E66C1EFFF66510001CCDF01011E
:103DB00066510D08D0E1036A65516225E96E6351D1
:103DC0000320EA6EEF6A0001000C01016B516D19CE
:103DD000800B6F6F6BAF05D06A1F6B1F6A2BD8B457
:103DE0006B2B6DAF05D06C1F6D1F6C2BD8B46D2B7A
:103DF0006A516C03F3CF01F0F4CF00F06D03F35080
:103E000000266B516C03F3500020026E6FAF05D09B
:103E1000011E021E012AD8B4022A000183EF1FF0FE
:103E20000101686B666B0A0E676F656B646B6251AC
:103E3000631104E1000E016E026EE8D06851682B38
:103E4000036A6225E96E63510320EA6EEFCF69F1E0
:103E500069512D080DE1010E666F6851682B036AE8
:103E60006225E96E63510320EA6EEFCF69F10DD050
:103E700069512B080AE16851682B036A6225E96ED3
:103E800063510320EA6EEFCF69F169512F08D8B072
:103E9000AFD069513908D8A0ABD06951300821E1C1
:103EA000036A68516225E96E63510320EA6EEF50A0
:103EB00078080AE0036A68516225E96E63510320BD
:103EC000EA6EEF5058080DE1100E676F682B6851CD
:103ED000682B036A6225E96E63510320EA6EEFCF17
:103EE00069F167510A0823E169512F081FE26951FE
:103EF00039081CE36B6B0A0E6A6F65C16DF164C112
:103F00006CF1000162D7300E0101695D0124646F1C
:103F1000000E0220656F6851682B036A6225E96E06
:103F200063510320EA6EEFCF69F1DED761D06751AC
:103F300010085EE16951600806E269517A0803E3FE
:103F40006951DF0B01D06951696F69512F0803E294
:103F50006951390806E2695140084AE26951460848
:103F600047E369512F0819E26951390816E36435AE
:103F70006A6F65356B6F6A376B376A376B376A37CD
:103F80006B37F00E6A17300E695D6A25016E000E00
:103F90006B2101C064F1656F16D064356A6F6535B9
:103FA0006B6F6A376B376A376B376A376B37F00E70
:103FB0006A17410E695D0A0F6A25016E000E6B21BA
:103FC00001C064F1656F6851682B036A6225E96E70
:103FD00063510320EA6EEF50696F600806E2695191
:103FE0007A0803E36951DF0B01D06951696FADD7DE
:103FF00067510A0807E1662D05D0641F651F642B11
:10400000D8B4652B64C101F065C102F0000119EF5D
:1040100020F0010E0101636F590E626F070E646F8D
:10402000000196DE010E0101636F590E626F0001FF
:10403000F7D602C061F101C060F1010160C101F079
:1040400061C102F00001000C006A016A01015551D2
:10405000D89056B100260032013256B30026003205
:10406000013256B500260032013256B70026003222
:10407000013256B900260032013256BB002600320A
:10408000013256BD00260032013256BF00260032F2
:1040900001320001BAEF20F00101536B516B0A0E9F
:1040A000526F506B4E514F1103E1000E016EC3D0A1
:1040B0005351532B036A4E25E96E4F510320EA6E8C
:1040C000EFCF54F154512D080DE1010E516F5351B2
:1040D000532B036A4E25E96E4F510320EA6EEFCF52
:1040E00054F10DD054512B080AE15351532B036A5C
:1040F0004E25E96E4F510320EA6EEFCF54F1545133
:104100002F08D8B090D054513908D8A08CD0545131
:10411000300821E1036A53514E25E96E4F510320C7
:10412000EA6EEF5078080AE0036A53514E25E96EB3
:104130004F510320EA6EEF5058080DE1100E526FF8
:10414000532B5351532B036A4E25E96E4F510320D5
:10415000EA6EEFCF54F152510A081DE154512F0875
:1041600019E25451390816E30A0E556F50C156F141
:1041700000016AD7300E0101545D0124506F535184
:10418000532B036A4E25E96E4F510320EA6EEFCFA1
:1041900054F1E4D748D05251100845E15451600819
:1041A00006E254517A0803E35451DF0B01D0545115
:1041B000546F54512F0803E25451390806E2545108
:1041C000400831E2545146082EE354512F080CE2C6
:1041D0005451390809E35039556FF00E5517300E18
:1041E000545D5525506F09D05039556FF00E551755
:1041F000410E545D0A0F5525506F5351532B036ADE
:104200004E25E96E4F510320EA6EEFCF54F1545121
:10421000600806E254517A0803E35451DF0B01D0E1
:104220005451546FC6D7512D04D052510A0801E1A0
:10423000506D50C101F000012EEF21F0010E01017F
:10424000636F480E626F050E646F000181DD010E21
:1042500001014F6F480E4E6F00011ED701C04DF196
:1042600001014DC101F00001000C0101426B416BE5
:104270000001BB9500EC11F0F20EF66E1F0EF76E0A
:10428000196AF2BE198EF29E15EC11F019BEF28E6B
:10429000C0DE02C046F101C045F1010146510708E8
:1042A00004E30BE14551D60808E24651060808E24E
:1042B000FF0A03E14551E10803E20001DDD70101F6
:1042C000D00E455D416F070E4659426FD89041C1EF
:1042D00042F1416B4237180EF66E200EF76E196AE6
:1042E000F2BE198EF29E000115EC11F019BEF28E8D
:1042F00090DE02C044F101C043F10101435302E1E9
:10430000445305E0445303E143510C0801E2E3D771
:1043100043374437433744374337443743374437C9
:1043200043374437E00E431743514113445142137E
:104330003C0EF66E200EF76E196AF2BE198EF29ED2
:10434000000115EC11F019BEF28E78DF01C047F1C3
:104350000101475303E047511F0801E2E9D74751E4
:104360004127000E422342C148F1496BAA6A130E4D
:10437000A96E48C1A8FFA69CA69EA684F250006E16
:10438000F29E0F01550EA76EAA0EA76EA682A6B2C8
:10439000FED7A6940050F212AA6A140EA96E41C16B
:1043A000A8FFA69CA69EA684F2CF00F0F29E550E12
:1043B000A76EAA0EA76EA682A6B2FED7A69400503C
:1043C000F2125E0EF66E200EF76E196AF2BE198EAC
:1043D000F29E000115EC11F019BEF28E42C148F1B7
:1043E0000101496B7C0EF66E200EF76E196AF2BE63
:1043F000198EF29E3B0E0201006F0001DBEC11F002
:1044000019BEF28E196AF2BE198EF29E48C1F5F1FC
:10441000370E0101F66F000146EC16F019BEF28E60
:10442000196AF2BE198EF29E41C1F5F1370E0101F3
:10443000F66F000146EC16F019BEF28E0D0E040068
:104440009EA8FDD7AD6E0A0E04009EA8FDD7AD6EE6
:1044500063EF37F093908A9093800400200E006EF3
:10446000002EFED700D093800101499181B049818F
:1044700004003B0E006E002EFED70000000E49B176
:10448000010E016E0001000C93908A90040000D090
:1044900000D001014A5309E093908A800400200E65
:1044A000006E002EFED700D008D093908A900400B2
:1044B000200E006E002EFED700D00400330E006EDA
:1044C000002EFED793800400090E006E002EFED74A
:1044D00000000001000C0101456B010E466F476BA7
:1044E000196AF2BE198EF29E000119EC15F019BE80
:1044F000F28E015203E1000E016E3CD1196AF2BE48
:10450000198EF29EF00E0101F66F000183EC15F09A
:1045100019BEF28E0400100E006E002EFED70101AF
:1045200046514008D8A01DD1000194DF01014891F7
:1045300001B0488100018EDF0101489301B048833A
:1045400048A108D048A306D0478547C101F0000123
:1045500011D1010148B198D048B396D03E51465D83
:1045600022E1010E465D006E0032003200321F0E65
:1045700000160050036ACF0F016E000E032201C027
:10458000E9FF03C0EAFF010E465D070B496F010E0C
:10459000006E4951016E04E0D8900036012EFCD720
:1045A0000050EF124AD046513E5D25E2010E465DB5
:1045B000006E0032003200321F0E00160050036AF7
:1045C000CF0F016E000E032201C0E9FF03C0EAFF16
:1045D000010E465D070B496F010E006E4951016ED9
:1045E00004E0D8900036012EFCD70050FF0AEF16E9
:1045F00046C145F122D0010E465D006E0032003208
:1046000000321F0E00160050036ACF0FE96E000E35
:104610000320EA6EEFCF49F1010E465D070B4A6FAA
:1046200049C100F04A51016E04E0D8900032012ED9
:10463000FCD700B002D046C145F1010E465D006EC8
:104640000032003200321F0E00160050036ACF0FF6
:10465000E96E000E0320EA6EEFCF49F1010E465DD0
:10466000070B4A6F49C100F04A51016E04E0D8902F
:104670000032012EFCD7000E00B0010E4A6F00017F
:1046800003DF0101462B6CD048A122D0010E465D0C
:10469000006E0032003200321F0E00160050036A16
:1046A000CF0F016E000E032201C0E9FF03C0EAFF35
:1046B000010E465D070B496F010E006E4951016EF8
:1046C00004E0D8900036012EFCD70050EF1222D023
:1046D000010E465D006E0032003200321F0E0016E1
:1046E0000050036ACF0F016E000E032201C0E9FFE4
:1046F00003C0EAFF010E465D070B496F010E006E15
:104700004951016E04E0D8900036012EFCD70050CC
:10471000FF0AEF16010E465D006E003200320032D5
:104720001F0E00160050036ACF0FE96E000E032023
:10473000EA6EEFCF49F1010E465D070B4A6F49C1A2
:1047400000F04A51016E04E0D8900032012EFCD7EF
:10475000000E00B0010E4A6F000196DE0101462BEB
:10476000DFD645C13EF13E5302E1478101D0478388
:1047700047C101F00001EBEF23F00101426B425110
:1047800009081AE3436B4351070814E34251080D2B
:10479000F350466B456F036A43514525016E465100
:1047A00003220150ED0FE96E000E0320EA6EEF6A5E
:1047B000432BE9D7422BE3D7010E426F0D0E0400C5
:1047C0009EA8FDD7AD6E0A0E04009EA8FDD7AD6E63
:1047D0003E6B000180D60150FB0FD8B0C6D0050F4C
:1047E000F1EF24F06A0EF66E1C0EF76E196AF2BE37
:1047F000198EF29E15EC11F019BEF28EF0D0010167
:1048000041531FE0196AF2BE198EF29E42C100F2B6
:10481000110E0201016F00013DEC11F019BEF28E84
:104820008D0EF66E1C0EF76E196AF2BE198EF29E90
:10483000040E0201006F0001DBEC11F019BEF28ED4
:104840000101436B4351070824E3010E425D080D4B
:10485000F350466B456F036A43514525016E46513F
:1048600003220150ED0F016E000E032203C046F13A
:10487000036A4351CF0FE96E000E0320EA6EEFCFBB
:1048800047F146C1EAFF01C0E9FF47C1EFFF432BF3
:10489000D9D7415305E0456B0001B3EC1DF0010190
:1048A0004491000162D0010141531FE0196AF2BE38
:1048B000198EF29E42C100F2110E0201016F000139
:1048C0003DEC11F019BEF28E950EF66E1C0EF76ED1
:1048D000196AF2BE198EF29E040E0201006F0001E9
:1048E000DBEC11F019BEF28E0101436B4351070856
:1048F00024E3010E425D080DF350466B456F036AD9
:1049000043514525016E465103220150ED0F016EC2
:10491000000E032203C046F1036A4351CF0FE96E34
:10492000000E0320EA6EEFCF47F146C1EAFF01C057
:10493000E9FF47C1EFFF432BD9D7415305E0456B52
:104940000001B3EC1DF00101422B448100010DD0A8
:104950009A0EF66E1C0EF76E196AF2BE198EF29E52
:1049600015EC11F019BEF28E3AD0010144A101D02C
:1049700030D7415333E0CE0EF66E1C0EF76E196A37
:10498000F2BE198EF29E000115EC11F019BEF28EE6
:104990001C0EF66E1D0EF76E196AF2BE198EF29E8F
:1049A00015EC11F019BEF28E640EF66E1D0EF76E48
:1049B000196AF2BE198EF29E15EC11F019BEF28E34
:1049C0003DDC01C043F101014351425D03E2FF0EB2
:1049D0003D6F03D0010E425D3D6F01D03D6B000184
:1049E000000CE824F76AF736FD0FF66E490EF72241
:1049F0000A00F550FA6E0800F550F96EE447FE47DC
:104A0000A6486A4950490101476B4751070818E316
:104A1000000E1CB0010E486F000E46B1010E481981
:104A200008E0D8901D321C32010E1C1AA00E1D1A6F
:104A300003D0D8901D321C32D8904633472BE5D78F
:104A40000001000C010141530EE06E0EF66E1E0EC9
:104A5000F76E196AF2BE198EF29E000115EC11F084
:104A600019BEF28E01013D3D01D00BD0196AF2BE94
:104A7000198EF29E0001BCEC15F019BEF28E2CD0FE
:104A80000101196AF2BE198EF29E000119EC15F0AF
:104A900019BEF28E0152D8A402D00101F2D704004F
:104AA000020E0101456F196AF2BE198EF29ED10EF7
:104AB000F76F0001B9EC10F019BEF28E0101452F1D
:104AC000F2D7196AF2BE198EF29ECC0EF66F000173
:104AD00083EC15F019BEF28E0400060E006E002E57
:104AE000FED7196AF2BE198EF29EAA0E0101F66F68
:104AF000000183EC15F019BEF28E0400060E006E64
:104B0000002EFED7196AF2BE198EF29E24EC16F022
:104B100019BEF28E01C0C7F00400060E006E002E12
:104B2000FED7196AF2BE198EF29E24EC16F019BE59
:104B3000F28E01C0C6F00400060E006E002EFED7F5
:104B4000196AF2BE198EF29E24EC16F019BEF28E8E
:104B500001C01AF01AC0C8F00101426B42510708A7
:104B600022E30400130E006E002EFED70000036A3D
:104B70004251BE0F016E000E032201C045F103C079
:104B800046F1196AF2BE198EF29E000124EC16F06D
:104B900019BEF28E46C1EAFF45C1E9FF01C0EFFF31
:104BA0000101422BDBD7196AF2BE198EF29E000179
:104BB00024EC16F019BEF28E01C044F104000C0E74
:104BC000006E002EFED700D0196AF2BE198EF29E3A
:104BD00024EC16F019BEF28E01C043F11D6A1C6A66
:104BE000AA0E0101466F00010EDFC7C046F10BDFC0
:104BF000C6C046F108DFC8C046F105DF0101426BBF
:104C00004251070810E3036A4251BE0FE96E000EDD
:104C10000320EA6EEFCF45F145C146F10001F3DE16
:104C20000101422BEDD71C1E1D1E4153D8B4DCD010
:104C3000200E04009EA8FDD7AD6E196AF2BE198E33
:104C4000F29EC7C0F5F1370EF66F000146EC16F084
:104C500019BEF28E200E04009EA8FDD7AD6E196A13
:104C6000F2BE198EF29EC6C0F5F1370E0101F66F45
:104C7000000146EC16F019BEF28E200E04009EA82C
:104C8000FDD7AD6E196AF2BE198EF29EC8C0F5F15D
:104C9000370E0101F66F000146EC16F019BEF28ED8
:104CA000200E04009EA8FDD7AD6E200E04009EA825
:104CB000FDD7AD6E200E04009EA8FDD7AD6E01019C
:104CC000426B425107081EE3036A4251BE0FE96E70
:104CD000000E0320EA6EEFCF45F1196AF2BE198E7D
:104CE000F29E45C1F5F1370EF66F000146EC16F065
:104CF00019BEF28E200E04009EA8FDD7AD6E0101F4
:104D0000422BDFD71DC045F1466B200E04009EA844
:104D1000FDD7AD6E200E04009EA8FDD7AD6E200E0F
:104D200004009EA8FDD7AD6E196AF2BE198EF29EE0
:104D300043C1F5F1370EF66F000146EC16F019BECF
:104D4000F28E200E04009EA8FDD7AD6E196AF2BE49
:104D5000198EF29E44C1F5F1370E0101F66F000184
:104D600046EC16F019BEF28E200E04009EA8FDD768
:104D7000AD6E280E04009EA8FDD7AD6E196AF2BE76
:104D8000198EF29E45C1F5F1370E0101F66F000153
:104D900046EC16F019BEF28E200E04009EA8FDD738
:104DA000AD6E196AF2BE198EF29E1CC0F5F1370E77
:104DB0000101F66F000146EC16F019BEF28E290EC5
:104DC00004009EA8FDD7AD6E0D0E04009EA8FDD771
:104DD000AD6E0A0E04009EA8FDD7AD6E0A0E04004B
:104DE0009EA8FDD7AD6E01010001000C04009EAA33
:104DF000FDD7AECF5EF101015E510001A3EC1EF0C4
:104E000001015E51390805E3300E5E5D016E0FD081
:104E10000ED05E51600806E25E517A0803E35E51EF
:104E2000DF0B01D05E51BF0F0A0F016E00D00001F1
:104E3000000CDCDF01C05DF1D9DF01C05CF10101D4
:104E40005C51DD0804E15DC101F007D006D05D5181
:104E5000100DF3505C25016E00D00001000C1D6A9E
:104E60001C6A0101415360E0A00EF66E1E0EF76E43
:104E7000196AF2BE198EF29E000115EC11F019BEEE
:104E8000F28ED7DF01C0AEF0AE518F0803E2010110
:104E9000EBD70001AF6BD80EF66E1E0EF76E196AD7
:104EA000F2BE198EF29E15EC11F019BEF28E030EB1
:104EB0000101426F42510A081FE30400A60E006E72
:104EC000002EFED7036A4251AE0F016E000E032280
:104ED00001C045F103C046F10001ABDF46C1EAFF66
:104EE00045C1E9FF01C0EFFF200E04009EA8FDD7D9
:104EF000AD6E0101422BDED70D0E04009EA8FDD73A
:104F0000AD6E0A0E04009EA8FDD7AD6E020EF66EC1
:104F10001F0EF76E196AF2BE198EF29E000115EC93
:104F200011F019BEF28E01013D3D01D00BD0196A7E
:104F3000F2BE198EF29E0001BCEC15F019BEF28E85
:104F40002CD00101196AF2BE198EF29E000119ECF3
:104F500015F019BEF28E0152D8A402D00101F2D789
:104F60000400020E0101456F196AF2BE198EF29E0D
:104F7000D10EF76F0001B9EC10F019BEF28E0101ED
:104F8000452FF2D7196AF2BE198EF29ECC0EF66F3B
:104F9000000183EC15F019BEF28E0400060E006EBF
:104FA000002EFED7196AF2BE198EF29E0F0E010175
:104FB000F66F000183EC15F019BEF28E0F0E0101A1
:104FC000466F000120DD0400060E006E002EFED7A5
:104FD000196AF2BE198EF29EAEC0F6F183EC15F09E
:104FE00019BEF28EAEC046F10EDD0400060E006E54
:104FF000002EFED7196AF2BE198EF29EAFC0F6F1EE
:1050000083EC15F019BEF28EAFC046F1FCDC030E46
:105010000101426F42510A082AE30400060E006EA5
:10502000002EFED7036A4251AE0FE96E000E032038
:10503000EA6EEFCF45F1196AF2BE198EF29E45C1B4
:10504000F6F1000183EC15F019BEF28E036A01013E
:105050004251AE0FE96E000E0320EA6EEFCF45F12C
:1050600045C146F10001CFDC0101422BD3D704003A
:10507000196AF2BE198EF29EC70EF76F0001B9ECE5
:1050800010F019BEF28E196AF2BE198EF29E24EC4F
:1050900016F019BEF28E01C043F10400060E006E38
:1050A000002EFED7196AF2BE198EF29E24EC16F07D
:1050B00019BEF28E01C044F11C1E1D1E0101415398
:1050C000D8B403D1000100EC11F01A0EF66E1F0ED9
:1050D000F76E196AF2BE198EF29E15EC11F019BE28
:1050E000F28E4C0EF66E1F0EF76E196AF2BE198E16
:1050F000F29E15EC11F019BEF28E196AF2BE198EED
:10510000F29EAEC0F5F1370E0101F66F000146ECDC
:1051100016F019BEF28E200E04009EA8FDD7AD6ECB
:10512000196AF2BE198EF29EAFC0F5F1370E010179
:10513000F66F000146EC16F019BEF28E200E040048
:105140009EA8FDD7AD6E200E04009EA8FDD7AD6EC3
:10515000200E04009EA8FDD7AD6E030E0101426F24
:1051600042510A081EE3036A4251AE0FE96E000E77
:105170000320EA6EEFCF45F1196AF2BE198EF29E56
:1051800045C1F5F1370EF66F000146EC16F019BE79
:10519000F28E200E04009EA8FDD7AD6E0101422BB9
:1051A000DFD70D0E04009EA8FDD7AD6E0A0E0400D9
:1051B0009EA8FDD7AD6E0A0E04009EA8FDD7AD6E69
:1051C0006E0EF66E1F0EF76E196AF2BE198EF29E03
:1051D000000115EC11F019BEF28E820EF66E1F0E54
:1051E000F76E196AF2BE198EF29E180E0201006F58
:1051F0000001DBEC11F019BEF28E196AF2BE198EB5
:10520000F29E44C1F5F1370E0101F66F000146EC44
:1052100016F019BEF28E196AF2BE198EF29E43C1C3
:10522000F5F1370E0101F66F000146EC16F019BEDC
:10523000F28E0D0E04009EA8FDD7AD6E0A0E04007E
:105240009EA8FDD7AD6E1DC045F10101466BA40EB1
:10525000F66E1F0EF76E196AF2BE198EF29E180EC8
:105260000201006F0001DBEC11F019BEF28E196A29
:10527000F2BE198EF29E45C1F5F1370E0101F66FAF
:10528000000146EC16F019BEF28E196AF2BE198EB4
:10529000F29E1CC0F5F1370E0101F66F000146ECDD
:1052A00016F019BEF28E0D0E04009EA8FDD7AD6E4D
:1052B0000A0E04009EA8FDD7AD6E0A0E04009EA83B
:1052C000FDD7AD6E92EC1EF001010001000C010152
:1052D0003D3D01D00BD0196AF2BE198EF29E00013D
:1052E000BCEC15F019BEF28E2CD00101196AF2BE89
:1052F000198EF29E000119EC15F019BEF28E0152C2
:10530000D8A402D00101F2D70400020E0101436FBC
:10531000196AF2BE198EF29ED10EF76F0001B9EC38
:1053200010F019BEF28E0101432FF2D7196AF2BEB6
:10533000198EF29ECC0EF66F000183EC15F019BEAB
:10534000F28E0400060E006E002EFED7196AF2BE21
:10535000198EF29E550E0101F66F000183EC15F0D7
:1053600019BEF28E0400060E006E002EFED7196ADA
:10537000F2BE198EF29EC7C0F6F183EC15F019BE8D
:10538000F28E196AF2BE198EF29E040E0101F86FB8
:10539000000101EC15F019BEF28E196AF2BE198EE9
:1053A000F29EC6C0F6F183EC15F019BEF28E196AB2
:1053B000F2BE198EF29E040E0101F86F000101EC9D
:1053C00015F019BEF28E196AF2BE198EF29EC8C08F
:1053D000F6F183EC15F019BEF28E196AF2BE198E41
:1053E000F29E040E0101F86F000101EC15F019BEE8
:1053F000F28E0101415371E0C60EF66E1F0EF76E7C
:10540000196AF2BE198EF29E000115EC11F019BE58
:10541000F28E196AF2BE198EF29E0A0E0101F86F21
:10542000000101EC15F019BEF28E196AF2BE198E58
:10543000F29E24EC16F019BEF28E01C042F1280E45
:1054400004009EA8FDD7AD6E196AF2BE198EF29EB9
:1054500042C1F5F1370E0101F66F000146EC16F07E
:1054600019BEF28E290E04009EA8FDD7AD6E200E47
:1054700004009EA8FDD7AD6E01014251AA080FE1BC
:10548000DA0EF66E1F0EF76E196AF2BE198EF29ED4
:10549000000115EC11F019BEF28E0ED00101E80EDC
:1054A000F66E1F0EF76E196AF2BE198EF29E00019B
:1054B00015EC11F019BEF28E080E0101436F196A46
:1054C000F2BE198EF29EFA0EF86F000101EC15F093
:1054D00019BEF28E0101432FF2D70001000C010129
:1054E000426B010E416F41510F0858E393908A902F
:1054F0000400030E446F196AF2BE198EF29EF20E7A
:10550000F76F0001B9EC10F019BEF28E0101442FC3
:10551000F2D793800400070E006E002EFED700D055
:10552000938081B01FD0720EF66E1D0EF76E196A51
:10553000F2BE198EF29E000115EC11F019BEF28E2A
:10554000020E0101446F196AF2BE198EF29EFA0E24
:10555000F86F000101EC15F019BEF28E0101442F25
:10556000F2D766D004006B0E006E002EFED700D07E
:105570009380439181A043810400196AF2BE198E81
:10558000F29EEF0EF76F0001B9EC10F019BEF28E2B
:10559000010143A101D0422B412BA5D7010E415D52
:1055A000446FA00EF66E1D0EF76E196AF2BE198ECC
:1055B000F29E090E0201006F0001DBEC11F019BE32
:1055C000F28E196AF2BE198EF29E44C100F21B0ED1
:1055D0000201016F00013DEC11F019BEF28EAB0E1D
:1055E000F66E1D0EF76E196AF2BE198EF29E070E48
:1055F0000201006F0001DBEC11F019BEF28E196A96
:10560000F2BE198EF29E42C100F21B0E0201016F22
:1056100000013DEC11F019BEF28E0D0E04009EA8A3
:10562000FDD7AD6E0A0E04009EA8FDD7AD6E010138
:1056300000011AEF38F0C00EF66E200EF76E196AF0
:10564000F2BE198EF29E15EC11F019BEF28EE60E26
:10565000F66E200EF76E196AF2BE198EF29E15ECE8
:1056600011F019BEF28EDAEC17F001013D3D01D0C8
:105670000BD0196AF2BE198EF29E0001BCEC15F037
:1056800019BEF28E2CD00101196AF2BE198EF29E5B
:10569000000119EC15F019BEF28E0152D8A402D007
:1056A0000101F2D70400020E0101DA6F196AF2BE9D
:1056B000198EF29ED10EF76F0001B9EC10F019BEF1
:1056C000F28E0101DA2FF2D7196AF2BE198EF29E1C
:1056D000CC0EF66F000183EC15F019BEF28E0400BB
:1056E000060E006E002EFED7196AF2BE198EF29ECB
:1056F000F00E0101F66F000183EC15F019BEF28E79
:105700000400060E006E002EFED7196AF2BE198E36
:10571000F29E0101F66B000183EC15F019BEF28ECA
:105720000400060E006E002EFED7196AF2BE198E16
:10573000F29E0101F66B000183EC15F019BEF28EAA
:105740000101416B4151970822E30400040E006EF1
:10575000002EFED70000036A4151420F016E010E78
:10576000032201C0DAF103C0DBF1196AF2BE198E1F
:10577000F29E000124EC16F019BEF28EDBC1EAFFA6
:10578000DAC1E9FF01C0EFFF0101412BDBD73D3D4D
:1057900001D030D0416B415107082BE30400060EC5
:1057A000006E002EFED7900E4125036A420F016E57
:1057B000010E032201C0DAF103C0DBF13D51080DF7
:1057C000F350DD6BDC6F036A4151DC25016EDD5166
:1057D00003220150ED0FE96E000E0320EA6EEFCFB9
:1057E000DCF1DBC1EAFFDAC1E9FFDCC1EFFF412BED
:1057F000D2D752D0196AF2BE198EF29E000119EC6E
:1058000015F019BEF28E0152D8A402D00101F2D7D0
:105810000400020E0101DA6F196AF2BE198EF29EBF
:10582000D10EF76F0001B9EC10F019BEF28E010134
:10583000DA2FF2D7196AF2BE198EF29E330EF66F86
:10584000000183EC15F019BEF28E900E0101416F3C
:105850004151970821E30400060E006E002EFED78A
:10586000036A4151420F016E010E032201C0DAF1B9
:1058700003C0DBF1196AF2BE198EF29E000124EC1E
:1058800016F019BEF28EDBC1EAFFDAC1E9FF01C0F2
:10589000EFFF0101412BDCD7416B4151970847E3F2
:1058A000300E04009EA8FDD7AD6E780E04009EA8B1
:1058B000FDD7AD6E196AF2BE198EF29E41C1F5F1A7
:1058C000370EF66F000146EC16F019BEF28E3A0E56
:1058D00004009EA8FDD7AD6E01014151DA6F010EA3
:1058E000DB6F036A4151420FE96E010E0320EA6E3D
:1058F000EFCFDCF1DBC1AAFFDAC1A9FFDCC1A8FF51
:10590000A69CA69EA684F250006EF29E0F01550E34
:10591000A76EAA0EA76EA682A6B2FED7A6940050C6
:10592000F2120001EAEC17F00101412BB6D7000E8C
:10593000F66E210EF76E196AF2BE198EF29E000104
:1059400015EC11F019BEF28E040E0101DA6F196A1E
:10595000F2BE198EF29EFA0EF86F000101EC15F0FE
:1059600019BEF28E0101DA2FF2D7000132EF38F0C2
:105970000101416B415197081BE3036A4151420FFA
:10598000E96E010E0320EA6E4151DD6F010EDE6FFC
:10599000F2CFDFF1F29EDEC1AAFFDDC1A9FFA69C16
:1059A000A69EA680A850DFBFF28EEF6E412BE2D7F5
:1059B000180EF66E210EF76E196AF2BE198EF29E5F
:1059C000000115EC11F019BEF28EDAEC17F0196A2D
:1059D000F2BE198EF29E19EC15F019BEF28E01522C
:1059E000F6E02A0E04009EA8FDD7AD6E196AF2BE3D
:1059F000198EF29E990E0101F66F000183EC15F0ED
:105A000019BEF28E0400200E006E002EFED700D0CC
:105A10000101416B41519708D8A0BCD0036A4151A4
:105A2000420FE96E010E0320EA6EEFCFDBF1196A37
:105A3000F2BE198EF29EDBC1F6F1000183EC15F087
:105A400019BEF28E0400100E006E002EFED7196AE9
:105A5000F2BE198EF29E24EC16F019BEF28E01C031
:105A6000DAF10400100E006E002EFED7036A010169
:105A70004151420FE96E010E0320EA6EEF50DA5DEC
:105A800031E1196AF2BE198EF29E770EF66F0001AF
:105A900083EC15F019BEF28EEAEC17F0196AF2BE2B
:105AA000198EF29E41C1F5F1370E0101F66F00012A
:105AB00046EC16F019BEF28E196AF2BE198EF29EED
:105AC000040E0101F86F000101EC15F019BEF28E11
:105AD000196AF2BE198EF29E24EC16F019BEF28EEF
:105AE00056D00101036A4151420FE96E010E0320B5
:105AF000EA6EEFCFDBF1196AF2BE198EF29E41C158
:105B0000F5F1370EF66F000146EC16F019BEF28E75
:105B10003A0E04009EA8FDD7AD6E196AF2BE198E2A
:105B2000F29EDBC1F5F1370E0101F66F000146EC84
:105B300016F019BEF28E200E04009EA8FDD7AD6EA1
:105B4000196AF2BE198EF29EDAC1F5F1370E010123
:105B5000F66F000146EC16F019BEF28E3B0EF66EA3
:105B6000210EF76E196AF2BE198EF29E040E020122
:105B7000006F0001DBEC11F019BEF28E0400200E64
:105B8000006E002EFED700D0010148D700010101B0
:105B9000412B40D7010EE16FE26BE36F0001FAEC9D
:105BA00017F0080E0101DB6F196AF2BE198EF29E22
:105BB000FA0EF86F000101EC15F019BEF28E01012A
:105BC000DB2FF2D700014BEF38F01B7E5EEF38F091
:105BD000010E0101AC6FAC51AB5D07E3A731AA33F5
:105BE000A933A833A733AC2BF6D7A7C100F0A8C1BF
:105BF00001F0A9C102F0AAC103F00001000C010EDE
:105C00000101AC6FAC51AB5D07E3AA35A737A837EC
:105C1000A937AA37AC2BF6D7A7C100F0A8C101F06D
:105C2000A9C102F0AAC103F00001000C120E01018B
:105C3000646F340E636F560E626F780E616F010EE3
:105C40005F6F5F510A0839E35F51040DF350036A37
:105C5000610F016E010E032201C0A1F103C0A2F188
:105C6000010E5F5D040DF350036A610FE96E010ED2
:105C70000320EA6EEFCFA3F1ECCFA4F1ECCFA5F1B6
:105C8000ECCFA6F1A6C1AAF1A5C1A9F1A4C1A8F1C2
:105C9000A3C1A7F1020EAB6F00019ADFA2C1EAFF18
:105CA000A1C1E9FF00C0EFFF01C0ECFF02C0ECFFA3
:105CB00003C0ECFF01015F2BC4D7F2CFA1F1F29E2C
:105CC000AA6A200EA96EA69CA69EA680A850A1BF77
:105CD000F28EA26FF2CFA3F1F29EAA6A210EA96EF4
:105CE000A69CA69EA680A850A3BFF28EA46F59C101
:105CF0008FF15AC190F1A2C18EF1A4C18DF19A0E1B
:105D0000946FBC0E936FDE0E926FF00E916FF2CF18
:105D1000A1F1F29EAA6A220EA96EA69CA69EA6805A
:105D2000A850A1BFF28EA26FA2C198F1FF0E976F8B
:105D3000FF0E966F800E956F9C6B9B6B9A6B996BA9
:105D4000A06B9F6B010E9E6FB80E9D6F670E0001DA
:105D5000DC6F450EDB6F230EDA6F010ED96FEF0E8D
:105D6000E06FCD0EDF6FAB0EDE6F890EDD6F980E2C
:105D7000E46FBA0EE36FDC0EE26FFE0EE16F100E01
:105D8000E86F320EE76F540EE66F760EE56FC30EC6
:105D9000EC6FD20EEB6FE10EEA6FF00EE96F0101CE
:105DA0005F6B5F514F08D8A014D35F510F0B606F2A
:105DB0005F510F08D8B087D06051040DF350036ACB
:105DC000610F016E010E032201C0A1F103C0A2F117
:105DD0000D0E60250F0B040DF350036A610FE96E81
:105DE000010E0320EA6EEFCFA3F1ECCFA4F1ECCFCC
:105DF000A5F1ECCFA6F1080E60250F0B040DF350B2
:105E0000036A610FE96E010E0320EA6EEFCF00F026
:105E1000ECCF01F0ECCF02F0ECCF03F00050A31B6D
:105E20000150A41B0250A51B0350A61B020E6025A7
:105E30000F0B040DF350036A610FE96E010E03208E
:105E4000EA6EEFCF00F0ECCF01F0ECCF02F0ECCF38
:105E500003F00050A31B0150A41B0250A51B0350CC
:105E6000A61B6051040DF350036A610FE96E010E29
:105E70000320EA6EEFCF00F0ECCF01F0ECCF02F0A0
:105E8000ECCF03F00050A31B0150A41B0250A51B34
:105E90000350A61BA6C1AAF1A5C1A9F1A4C1A8F1EE
:105EA000A3C1A7F1010EAB6F0001A9DEA2C1EAFFF9
:105EB000A1C1E9FF00C0EFFF01C0ECFF02C0ECFF91
:105EC00003C0ECFF01015F51130802E2000E01D094
:105ED000010E010BD8B494D0DCC0AAF1DBC0A9F14B
:105EE000DAC0A8F1D9C0A7F1050EAB6F000187DEBB
:105EF00003C0A4F102C0A3F101C0A2F100C0A1F14E
:105F0000DD51E1150101A56F0001DE51E21501012E
:105F1000A66F0001DF51E3150101A76F0001E051F9
:105F2000E4150101A86FDDC0A9F10101A91FDEC0C0
:105F3000AAF10101AA1FDFC0ABF10101AB1FE0C054
:105F4000ACF10101AC1FA9510001E515006E010182
:105F5000AA510001E615016E0101AB510001E715E0
:105F6000026E0101AC510001E815036E0050010101
:105F7000A511006E0150A611016E0250A711026E0C
:105F80000350A811036E0050A1270150A223025014
:105F9000A3230350A4230001E9510101A12700011B
:105FA000EA510101A2230001EB510101A3230001E9
:105FB000EC510101A4236051040DF350036A610FF9
:105FC000E96E010E0320EA6EEFCF00F0ECCF01F096
:105FD000ECCF02F0ECCF03F00050A1270150A22338
:105FE0000250A3230350A423990EA1255B6F790EC1
:105FF000A2215C6F820EA3215D6F5A0EA4215E6FF9
:106000005F51130802E3000E01D0010EA16F5F5132
:10601000270802E2000E01D0010EA11578E0DCC0D5
:10602000AAF1DBC0A9F1DAC0A8F1D9C0A7F1050E29
:10603000AB6F0001E4DD03C0A4F102C0A3F101C015
:10604000A2F100C0A1F1DD51E1190101A56F00012C
:10605000DE51E2190101A66F0001DF51E3190101D0
:10606000A76F0001E051E4190101A86FA5510001DB
:10607000E519006E0101A6510001E619016E01014A
:10608000A7510001E719026E0101A8510001E819AA
:10609000036E00500101A1270150A2230250A32347
:1060A0000350A4230001E9510101A1270001EA5195
:1060B0000101A2230001EB510101A3230001EC51D6
:1060C0000101A4236051040DF350036A610FE96ECE
:1060D000010E0320EA6EEFCF00F0ECCF01F0ECCF21
:1060E00002F0ECCF03F00050A1270150A223025090
:1060F000A3230350A423A10EA1255B6FEB0EA221C5
:106100005C6FD90EA3215D6F6E0EA4215E6F5F518F
:10611000270802E3000E01D0010EA16F5F513B087A
:1061200002E2000E01D0010EA115D8B494D0DCC05B
:10613000AAF1DBC0A9F1DAC0A8F1D9C0A7F1050E18
:10614000AB6F00015CDD03C0A4F102C0A3F101C08C
:10615000A2F100C0A1F1DD51E1150101A56F00011F
:10616000DE51E2150101A66F0001DF51E3150101C7
:10617000A76F0001E051E4150101A86F0001DD5196
:10618000E515006EDE51E615016EDF51E715026E72
:10619000E051E815036E00500101A5130150A6134C
:1061A0000250A7130350A8130001E151E515006E3A
:1061B000E251E615016EE351E715026EE451E81570
:1061C000036E00500101A511006E0150A611016E71
:1061D0000250A711026E0350A811036E0050A127B0
:1061E0000150A2230250A3230350A4230001E9512C
:1061F0000101A1270001EA510101A2230001EB5195
:106200000101A3230001EC510101A4236051040DFD
:10621000F350036A610FE96E010E0320EA6EEFCFBF
:1062200000F0ECCF01F0ECCF02F0ECCF03F0005027
:10623000A1270150A2230250A3230350A423DC0E64
:10624000A1255B6FBC0EA2215C6F1B0EA3215D6FAD
:106250008F0EA4215E6F5F513B0802E3000E01D058
:10626000010EA16F5F514F0802E2000E01D0010E36
:10627000A11578E0DCC0AAF1DBC0A9F1DAC0A8F171
:10628000D9C0A7F1050EAB6F0001B9DC03C0A4F1C2
:1062900002C0A3F101C0A2F100C0A1F1DD51E119DA
:1062A0000101A56F0001DE51E2190101A66F000195
:1062B000DF51E3190101A76F0001E051E419010169
:1062C000A86FA5510001E519006E0101A65100015A
:1062D000E619016E0101A7510001E719026E0101E3
:1062E000A8510001E819036E00500101A1270150D7
:1062F000A2230250A3230350A4230001E95101016A
:10630000A1270001EA510101A2230001EB51010183
:10631000A3230001EC510101A4236051040DF350AB
:10632000036A610FE96E010E0320EA6EEFCF00F001
:10633000ECCF01F0ECCF02F0ECCF03F00050A1273E
:106340000150A2230250A3230350A423D60EA1255B
:106350005B6FC10EA2215C6F620EA3215D6FCA0E3E
:10636000A4215E6FE8C0ECF0E7C0EBF0E6C0EAF015
:10637000E5C0E9F0E4C0E8F0E3C0E7F0E2C0E6F031
:10638000E1C0E5F0E0C0AAF1DFC0A9F1DEC0A8F1EC
:10639000DDC0A7F1020EAB6F00011ADC03C0E4F010
:1063A00002C0E3F001C0E2F000C0E1F0DCC0E0F0C8
:1063B000DBC0DFF0DAC0DEF0D9C0DDF05EC1DCF0BA
:1063C0005DC1DBF05CC1DAF05BC1D9F001015F2B8C
:1063D000E8D40001E8EF32F000EC11F0F2CF59F10F
:1063E000F29EAA6A200EA96EA69CA69EA680A85020
:1063F000010159BFF28E5A6FF2CF5BF1F29EAA6A89
:10640000210EA96EA69CA69EA680A8505BBFF28E08
:106410005C6F5AC15EF15CC15DF1F2CF5FF1F29E3B
:10642000AA6A220EA96EA69CA69EA680A8505FBF4F
:10643000F28E606F040EF66E190EF76E196AF2BED8
:10644000198EF29E150E0201006F0001DBEC11F0B7
:1064500019BEF28E100EE96E196AF2BE198EF29E06
:106460005EC1FEF15DC1FDF17FEC11F019BEF28E4F
:106470001C0EF66E190EF76E196AF2BE198EF29E98
:106480000D0E0201006F0001DBEC11F019BEF28E5F
:10649000196AF2BE198EF29E60C100F21B0E020153
:1064A000016F00013DEC11F019BEF28E0D0E0400DB
:1064B0009EA8FDD7AD6E0A0E04009EA8FDD7AD6E56
:1064C0000A0E04009EA8FDD7AD6E300EF66E190EB2
:1064D000F76E196AF2BE198EF29E15EC11F019BE14
:1064E000F28E7E0EF66E190EF76E196AF2BE198ED6
:1064F000F29E15EC11F019BEF28EF2CF59F1F29E18
:10650000AA6A100EA96EA69CA69EA680A85001019C
:1065100059BFF28E5A6FF2CF5BF1F29EAA6A110E4A
:10652000A96EA69CA69EA680A8505BBFF28E5C6F4B
:106530005AC144F15CC143F1CC0EF66E190EF76EF0
:10654000196AF2BE198EF29E130E0201006F00014D
:10655000DBEC11F019BEF28E100EE96E196AF2BE74
:10656000198EF29E44C1FEF143C1FDF17FEC11F0A2
:1065700019BEF28E0D0E04009EA8FDD7AD6E0A0E58
:1065800004009EA8FDD7AD6E0A0E04009EA8FDD79C
:10659000AD6EE60EF66E190EF76E196AF2BE198E22
:1065A000F29E15EC11F019BEF28E09EC20F002C03B
:1065B00042F101C041F10101415303E1425301E1C4
:1065C000C8D142C15AF141C159F1000116EF2EF074
:1065D0001E0EF66E1A0EF76E196AF2BE198EF29E34
:1065E00015EC11F019BEF28E480EF66E170EF76E0E
:1065F000196AF2BE198EF29E15EC11F019BEF28ED8
:106600004C0EF66E1A0EF76E196AF2BE198EF29ED5
:1066100015EC11F019BEF28E19EC27F001C059F1FA
:1066200019EC27F001C05AF119EC27F001C05BF119
:1066300019EC27F059C148F15AC147F15BC146F145
:1066400001C045F119EC27F001C059F119EC27F010
:1066500001C05AF119EC27F001C05BF119EC27F0E9
:1066600059C14CF15AC14BF15BC14AF101C049F12A
:1066700019EC27F001C059F119EC27F001C05AF1CB
:1066800019EC27F001C05BF119EC27F059C150F16A
:106690005AC14FF15BC14EF101C04DF119EC27F029
:1066A00001C059F119EC27F001C05AF119EC27F09B
:1066B00001C05BF119EC27F059C154F15AC153F1F3
:1066C0005BC152F101C051F119EC27F001C059F141
:1066D00019EC27F001C05AF119EC27F001C05BF169
:1066E00019EC27F059C158F15AC157F15BC156F165
:1066F00001C055F1D9510101455DD8A40CD100016B
:10670000DA510101465DD8A406D10001DB51010137
:10671000475DD8A400D10001DC510101485DD8A437
:10672000FAD00001DD510101495DD8A4F4D0000187
:10673000DE5101014A5DD8A4EED00001DF51010114
:106740004B5DD8A4E8D00001E05101014C5DD8A414
:10675000E2D00001E15101014D5DD8A4DCD000017F
:10676000E25101014E5DD8A4D6D00001E3510101F0
:106770004F5DD8A4D0D00001E4510101505DD8A4F0
:10678000CAD00001E5510101515DD8A4C4D0000177
:10679000E6510101525DD8A4BED00001E7510101CC
:1067A000535DD8A4B8D00001E8510101545DD8A4CC
:1067B000B2D00001E9510101555DD8A4ACD000016F
:1067C000EA510101565DD8A4A6D00001EB510101A8
:1067D000575DD8A4A0D00001EC510101585DD8A4A8
:1067E0009AD0435141274451422342C159F15A6B37
:1067F000AA6A100EA96E59C1A8FFA69CA69EA684DF
:10680000F250006EF29E0F01550EA76EAA0EA76EF3
:10681000A682A6B2FED7A6940050F212AA6A110E62
:10682000A96E41C1A8FFA69CA69EA684F2CF00F047
:10683000F29E550EA76EAA0EA76EA682A6B2FED72E
:10684000A6940050F212F2CF59F1F29EAA6A220EDB
:10685000A96EA69CA69EA680A850010159BFF28EE3
:10686000010F5A6FAA6A220EA96E5AC1A8FFA69CF0
:10687000A69EA684F250006EF29E0F01550EA76EE2
:10688000AA0EA76EA682A6B2FED7A6940050F21258
:10689000520EF66E1A0EF76E196AF2BE198EF29E3D
:1068A0002B0E0201006F0001DBEC11F019BEF28E1D
:1068B000100EE96E196AF2BE198EF29E44C1FEF105
:1068C00043C1FDF17FEC11F019BEF28E800EF66E21
:1068D0001A0EF76E196AF2BE198EF29E040E0201AC
:1068E000006F0001DBEC11F019BEF28E100EE96EA4
:1068F000196AF2BE198EF29E42C1FEF141C1FDF14C
:106900007FEC11F019BEF28E2E0E04009EA8FDD76A
:10691000AD6E0ED001018A0EF66E1A0EF76E196A70
:10692000F2BE198EF29E000115EC11F019BEF28E26
:10693000080E0101596F196AF2BE198EF29EFA0E05
:10694000F86F000101EC15F019BEF28E0101592F0C
:10695000F2D7000174EF38F0FF0E01013D6F416B7B
:106960004151070819E3036A4151ED0F016E000E12
:10697000032203C043F1036A4151CF0FE96E000EB9
:106980000320EA6EEFCF44F143C1EAFF01C0E9FF03
:1069900044C1EFFF412BE4D70001000C41C1AEF030
:1069A000AF6BAA0EB16F550EB26F020EAE25036A21
:1069B0001E0FE96E000E0320EA6EEFCFB3F0030E58
:1069C000AE25036A1E0FE96E000E0320EA6EEFCFBC
:1069D000B4F0040EAE25036A1E0FE96E000E03200C
:1069E000EA6EEFCFB5F0050EAE25036A1E0FE96E15
:1069F000000E0320EA6EEFCFB6F0060EAE25036A56
:106A00001E0FE96E000E0320EA6EEFCFB7F0070EFF
:106A1000AE25036A1E0FE96E000E0320EA6EEFCF6B
:106A2000B8F0000C41C1AEF0AF6B036AAE511E0F5F
:106A3000E96E000E0320EA6EEFCFB1F0010EAE2535
:106A4000036A1E0FE96E000E0320EA6EEFCFB2F06C
:106A5000020EAE25036A1E0FE96E000E0320EA6ED9
:106A6000EFCFB3F0030EAE25036A1E0FE96E000EE2
:106A70000320EA6EEFCFB4F0040EAE25036A1E0FBA
:106A8000E96E000E0320EA6EEFCFB5F0050EAE25DD
:106A9000036A1E0FE96E000E0320EA6EEFCFB6F018
:106AA000AA0EB76F550EB86F000CF86AD09E078E0D
:106AB000EA6AE96AB8862A0EAF6E000EB06EA60EBC
:106AC000AC6E900EAB6EBB91FF0EBC6FBD6BBB93FB
:106AD000BB95D86BD76B01013D6FC150C00B0F093F
:106AE000C16E070EB46E0001C96BCA6B810ECF6F09
:106AF000D06BD16BD26B010ED36F300ED46F100EF2
:106B0000D56FD66BD190C150C00B0F09C16EC2902A
:106B1000C69A949A94889496010EC66E000EC76E1B
:106B2000D190810ED56ECD6A000ECA6E000ECB6E6E
:106B3000070EB46E9250926E0400100E006E002E7E
:106B4000FED7B450A19CB56ABAEC17F0196AF2BE30
:106B5000198EF29E640E0101F86F000101EC15F030
:106B600019BEF28EBDEC17F0F2CF41F1F29EAA6A87
:106B7000240EA96EA69CA69EA680A850010141BF26
:106B8000F28E1B6E0001BFEF17F0196AF2BE198E6C
:106B9000F29E95EC14F019BEF28ED76AD66AF29482
:106BA000F28AC00EF212D18004009EAAFDD7AECFA9
:106BB0003FF101013F51600806E23F517A0803E3CB
:106BC0003F51DF0B01D03F513F6F40513F5D05E02A
:106BD0000001D86B010ED76F04D00001D72BD8B4B9
:106BE000D82BBAEC17F001013F51310A00013CE00B
:106BF000030A5DE0010AD8B47ED0070AD8B49FD05A
:106C0000010AD8B4C0D0030AD8B4E1D0770AD8B406
:106C100002D1030AD8B425D10B0AD8B44AD10A0A42
:106C2000D8B461D1060AD8B47FD1030AD8B49BD1B5
:106C3000010AD8B4B5D10F0AD8B4CFD1040AD8B458
:106C4000EED1020AD8B403D2010AD8B419D21F0A6D
:106C5000D8B42CD2010AD8B43FD2090AD8B450D241
:106C60000B0AD8B45AD251D3BC3D01D059D3F29AB1
:106C7000310E04009EA8FDD7AD6E0D0E04009EA837
:106C8000FDD7AD6E0A0E04009EA8FDD7AD6E0101C2
:106C9000416B0001FFEC18F0196AF2BE198EF29EEA
:106CA00095EC14F019BEF28EF294F28A39D3BC3D01
:106CB00001D036D3F29A320E04009EA8FDD7AD6EF5
:106CC0000D0E04009EA8FDD7AD6E0A0E04009EA80E
:106CD000FDD7AD6E010E0101416F0001FFEC18F010
:106CE000196AF2BE198EF29E95EC14F019BEF28E5E
:106CF000F294F28A15D3BC3D01D012D3F29A330E2E
:106D000004009EA8FDD7AD6E0D0E04009EA8FDD711
:106D1000AD6E0A0E04009EA8FDD7AD6E020E0101F5
:106D2000416F0001FFEC18F0196AF2BE198EF29E55
:106D300095EC14F019BEF28EF294F28AF1D2BC3DB9
:106D400001D0EED2F29A340E04009EA8FDD7AD6EAB
:106D50000D0E04009EA8FDD7AD6E0A0E04009EA87D
:106D6000FDD7AD6E030E0101416F0001FFEC18F07D
:106D7000196AF2BE198EF29E95EC14F019BEF28ECD
:106D8000F294F28ACDD2BC3D01D0CAD2F29A350E2D
:106D900004009EA8FDD7AD6E0D0E04009EA8FDD781
:106DA000AD6E0A0E04009EA8FDD7AD6E040E010163
:106DB000416F0001FFEC18F0196AF2BE198EF29EC5
:106DC00095EC14F019BEF28EF294F28AA9D2BC3D71
:106DD00001D0A6D2F29A360E04009EA8FDD7AD6E61
:106DE0000D0E04009EA8FDD7AD6E0A0E04009EA8ED
:106DF000FDD7AD6E050E0101416F0001FFEC18F0EB
:106E0000196AF2BE198EF29E95EC14F019BEF28E3C
:106E1000F294F28A85D2BC3D01D082D2F29A410E20
:106E200004009EA8FDD7AD6E010E0101416F000167
:106E30003BEF1EF0BDEC17F092EC1EF0196AF2BEAB
:106E4000198EF29E95EC14F019BEF28EBC51FE081C
:106E500005E1FF0E01013D6F0001BD6FF294F28A62
:106E60005FD2BC3D01D05CD2F29A420E04009EA8D3
:106E7000FDD7AD6E00EC11F0196AF2BE198EF29ECC
:106E8000010E0101EF6FF06B00016BEC16F019BE03
:106E9000F28E92EC1EF0196AF2BE198EF29E95ECFB
:106EA00014F019BEF28EBC51FE0802E0F294F28A90
:106EB00037D2F29A450E04009EA8FDD7AD6E00ECC5
:106EC00011F035EF21F092EC1EF0196AF2BE198E26
:106ED000F29E95EC14F019BEF28EBC51FE0802E051
:106EE000F294F28A1DD2BC3D01D01AD2BBB101D0BE
:106EF00017D2F29A430E04009EA8FDD7AD6E010E84
:106F00000101416F0001BDEC23F0BDEC17F092ECE4
:106F10001EF0196AF2BE198EF29E95EC14F019BE9D
:106F2000F28EF294F28AFCD1BC3D01D0F9D1F29AF2
:106F3000450E04009EA8FDD7AD6E010E0101416F04
:106F4000000122EC25F092EC1EF0196AF2BE198EB7
:106F5000F29E95EC14F019BEF28EBC51FE0802E0D0
:106F6000F294F28ADDD1BC3D01D0DAD1F29A460E1C
:106F700004009EA8FDD7AD6E010E0101416F000116
:106F80002FEC27F0196AF2BE198EF29E95EC14F0E0
:106F900019BEF28EBC51FE0802E0F294F28AC0D112
:106FA000BC3D01D0BDD1F29A470E04009EA8FDD78A
:106FB000AD6E010E0101416F000167EC29F0196A05
:106FC000F2BE198EF29E95EC14F019BEF28EBC51F1
:106FD000FE0802E0F294F28AA3D1F29A480E04006D
:106FE0009EA8FDD7AD6E00EC11F0196AF2BE198EA5
:106FF000F29E010E0101EF6FF06F00016BEC16F0D5
:1070000019BEF28E92EC1EF0196AF2BE198EF29E33
:1070100095EC14F019BEF28EF294F28A81D1BC3D47
:1070200001D07ED1F29A4C0E04009EA8FDD7AD6E21
:107030006FEF2AF092EC1EF0196AF2BE198EF29EE2
:1070400095EC14F019BEF28EF294F28A69D1BC3D2F
:1070500001D066D1F29A4E0E04009EA8FDD7AD6E07
:107060001BEF2BF0196AF2BE198EF29E95EC14F00C
:1070700019BEF28EBC51FE0802E0F294F28A50D1A1
:10708000BC3D01D04DD1F29A4F0E04009EA8FDD711
:10709000AD6EB8EF2CF0196AF2BE198EF29E95EC27
:1070A00014F019BEF28EF294F28A3AD1F29A500E8E
:1070B00004009EA8FDD7AD6EE5EF2DF092EC1EF01A
:1070C000196AF2BE198EF29E95EC14F019BEF28E7A
:1070D000F294F28AD18024D1F29A470E04009EA83D
:1070E000FDD7AD6EECEF31F0196AF2BE198EF29E4B
:1070F00095EC14F019BEF28EF294F28AD18010D180
:10710000F29ABB71196AF2BE198EF29E95EC14F0D8
:1071100019BEF28EF294F28A03D1BC3D01D000D1A7
:10712000F29A530E04009EA8FDD7AD6E0101416B8B
:107130000001BDEC23F010DC196AF2BE198EF29E3C
:107140000101EF6BF06B00016BEC16F019BEF28ED3
:107150000101416B0001BDEC23F0196AF2BE198EEA
:10716000F29E5A0E0101F86F000101EC15F019BEF4
:10717000F28EACEC34F0196AF2BE198EF29E010167
:10718000EF6BF06B00016BEC16F019BEF28E050E82
:107190000101416F196AF2BE198EF29E5F0EF86FFF
:1071A000000101EC15F019BEF28E0101412FF2D75A
:1071B000200E416F0001CEEC34F00101416B000163
:1071C0002FEC27F00101416B000122EC25F00101B9
:1071D000416B000167EC29F0196AF2BE198EF29E2C
:1071E0000C0E0101F86F000101EC15F019BEF28ED2
:1071F000380E0101416F000115DC0101416B0001F6
:107200002FEC27F00101416B000122EC25F0010178
:10721000416B000167EC29F0196AF2BE198EF29EEB
:107220000E0E0101F86F000101EC15F019BEF28E8F
:10723000400E0101416F0001CEEC34F00101416BC1
:1072400000012FEC27F00101416B000122EC25F039
:107250000101416B000167EC29F0196AF2BE198E39
:10726000F29E0E0E0101F86F000101EC15F019BE3F
:10727000F28E580E0101416F000112EC35F0010150
:10728000416B00012FEC27F00101416B000122EC62
:1072900025F00101416B000167EC29F0196AF2BE8B
:1072A000198EF29E1F0E0101F86F000101EC15F01E
:1072B00019BEF28E0101416B0001BDEC23F0196A89
:1072C000F2BE198EF29E5A0E0101F86F000101EC18
:1072D00015F019BEF28EACEC34F0196AF2BE198EBC
:1072E000F29E0101EF6BF06B00016BEC16F019BE22
:1072F000F28E196AF2BE198EF29E95EC14F019BE48
:10730000F28EF294F28AD1800BD00D0E04009EA86A
:10731000FDD7AD6E0A0E04009EA8FDD7AD6E00D05D
:0C732000BDEC17F03FC140F13FD403006A
:020000040030CA
:0E00000000C20E1E00858100000007A0070050
:00000001FF
